:106BFE000000050200000301FA0400EF0500030A7D
:106C0E000A5A0B001E0C00FA0D00030E00040F01B1
:106C1E0064100096120132130AFA14010217010AC7
:106C2E001801EF1905321A010A1B01EF1C05321F5C
:106C3E00FFFF20FFFF23011E2400642A00FA2B0011
:106C4E00FA2C50782D003C2E0046300064325078DD
:106C5E003301013432FF3501643601643701503897
:106C6E000A643A00033B00043C00643E003C3F00D3
:106C7E000140002D411450420A5A430AC8440532BD
:106C8E004500B44600FA4900024B00014C00FA5090
:106C9E000202510596520A32530B46540A96570574
:106CAE0046590A465A32FA5B010A5C0A325E000AFB
:106CBE005F00646200FE64021C67FFFF68010169E9
:106CCE0001016A05966B00006C32FF6D00047300C3
:106CDE00007400007801327901327EFFFF81FFFFE0
:106CEE0084FFFF8800028A00019D0A969E00019F84
:106CFE00FFFFA0FFFFA2000AA3003BA40064A500B3
:106D0E0064A6FFFFA7FFFFA8FFFFA9FFFF01013C3D
:106D1E001500002F003C47003C4804045602044E68
:106D2E00FFFF58000261FFFF6600028500AF86007C
:106D3E00018700FA89010A990004A100FAFAFAFA09
:106D4E0001013C1500002F1E3C47013C480404562F
:106D5E0002044EFFFF58000261FFFF66000285002D
:106D6E00AF8600018700FA89010A990000A1000090
:106D7E00FAFAFA0065006F00790083008D00970023
:106D8E00A100AC00B600C000CA00D400DE00E800CE
:106D9E00F2005800600068007000780080008800E3
:106DAE0090009800A000A800B000B800C100C80074
:106DBE00D000D800DF00E600EE00F60041004700EC
:106DCE004D00530059005F0065006C0071007700A4
:106DDE007D00830089008F0095009B00A200A70014
:106DEE00AC00B200B900C000C500CA00D200D50088
:076DFE00DD00E100E700EFFA
:103D750075A71085F97285FA737E017F00E57312C8
:103D85006F17E5722FFF50010E8E588F5922900044
:103D950084E0FE900079E0D39E5012900084E0FE0E
:103DA500900079E0F4042E90004AF080129000848F
:103DB500E0243CFE900079E0F4042E90004AF09057
:103DC500004AE0B41E06741F90004AF090004AE0D5
:103DD500B41D06741C90004AF090004AE0600790FC
:103DE500004AE0B43C0690004A7401F090004AE0B5
:103DF500D3941E400D90004AE0C3941E90004CF0F1
:103E0500800A90004AE0241E90004CF02290008425
:103E1500E0FE90007AE0D39E5012900084E0FE9080
:103E2500007AE0F4042E90004BF08012900084E0BC
:103E3500243CFE90007AE0F4042E90004BF09000B4
:103E45004BE0B41E06741F90004BF090004BE0B49D
:103E55001D06741C90004BF090004BE0600790002D
:103E65004BE0B43C0690004B7401F090004BE0D35E
:103E7500941E400D90004BE0C3941E90004DF080C1
:103E85000A90004BE0241E90004DF022E50C90674F
:103E9500EDF8282873023F31A22DB34008E5B5445B
:103EA50008F5B58006E5B554F7F5B5807FA22DB3C5
:103EB5004008E5B54402F5B58006E5B554FDF5B510
:103EC500806AA22D92A28064A22D92A1805EA22D6D
:103ED50092878058A22D92908052A22DB34008E57A
:103EE500B54410F5B58006E5B554EFF5B5803DA2AE
:103EF5002DB34008E5B54420F5B58006E5B554DF9A
:103F0500F5B58028A22DB34008E5B54440F5B58048
:103F150006E5B554BFF5B58013A22DB34008E5B548
:0C3F25004480F5B58006E5B5547FF5B585
:1067ED00023E9A023E9D023EB2023EC7023ECD02DD
:1067FD003ED3023ED9023EDF023EF4023F09023F84
:01680D001E6C
:103F310022745290015AF0745890015BF0743890D9
:103F4100015CF0742090015DF0743690015EF074B4
:103F51003090015FF0742D900160F0743290016136
:103F6100F07420900162F07432900163F074529009
:103F71000164F0746F900165F07474900166F074DF
:103F81006F900167F07472900168F022900891E0DF
:103F9100FEA3E0FF741DD39F74019E400C906BFE45
:103FA100120048E493F599802E90F802E493B40549
:103FB10014900891E0FEA3E0FF906C31120048E4F8
:103FC10093F5998012900891E0FEA3E0FF906BFEBB
:103FD100120048E493F599900891126F2590089189
:103FE100E0FEA3E0FFEFB45007EEB40103754C000F
:103FF10022AE58AF5974068E048F05FF126F078CDD
:104001005A8D5BAE58AF5974068E048F05FF126F3F
:10401100328C588D59E559455860137406C395592A
:10402100FFE49558FE8E588F59785A126F6AE572DF
:10403100A85AB80015D3955B4010E572C3955BFF94
:10404100E4955AFE8E5A8F5B8010E572243CC3952D
:104051005BFFE4955AFE8E5A8F5BAE5AAF5B743BA1
:104061006F4E6006743C6F4E701AAE5AAF5B743B74
:104071006F4E70057572018003757202755B3A753A
:104081005A00800375720022900097E0B40104C2C7
:10409100068002D2069000D5E075F0D7A4FFAEF0FD
:1040A100740A8E048F05FF126F07900885ECF0A348
:1040B100EDF09000D5E075F02BA4FFAEF090001A62
:1040C100EEF0A3EFF07E017F00900093E0126F17F6
:1040D1009000D6E08E048F05FF126F07740AFF125D
:1040E1006F078D5F9000DFE075F0D7A4FFAEF0742D
:1040F1000A8E048F05FF126F07900889ECF0A3ED7B
:10410100F09000E1E060139000E1E0F5F0741684B6
:10411100FF7E00EF9008E7F0800674649008E7F0F6
:104121009000D7E0900077F0900125E0FE9000D359
:10413100E08E0088F0A4FFAEF0EF9008F0F0900060
:10414100FEE075F013A4FDACF090003EECF0A3EDA1
:10415100F0A21AB3401690016FE0700C900170E06C
:104161007006900171E060028002C21A90016FE056
:10417100B4300F900170E0B44708900171E0643BE6
:1041810060028004D21B8002C21B9000BEE0B40317
:10419100089000E9E064026002800874009000E980
:1041A100F0D219900090E0FE9008F1E06E601A756F
:1041B10099E612019C74AB900051F01206DA750970
:1041C1006475080012062480FE900088E070067471
:1041D100009000BDF090007BE0FE9000BDE0B506D0
:1041E1003390007DE0FE9000DBE0B5062790007E75
:1041F100E0FE900090E0B5061B90007CE0FE900090
:10420100D9E0B5060F90007FE0FE900109E06E70E5
:1042110003024345740A90010CF09000D9E0B40305
:104221000674029000D9F0900090E0B40106740089
:10423100900090F0900090E0B4020674009000DBD2
:10424100F0900090E0B4030674009000E8F0900054
:10425100DBE0D394014014741990010EF0740090C6
:1042610006D1F074009006D2F0800C740090010E1B
:10427100F074199006D1F09000BDE06014741A90AA
:1042810000A4F074009006D5F074009006D6F0807A
:104291000C74009000A4F0741A9006D5F09000BD43
:1042A100E0B40214741B9000A5F074009006E9F0CC
:1042B10074009006EAF0800C74009000A5F0741B65
:1042C1009006E9F0900109E060147407900781F00D
:1042D10074009006E1F074009006E2F0800C740026
:1042E100900781F074079006E1F07401900779F06E
:1042F100740290077AF0740390077BF074049007BE
:104301007CF07415900771F07416900772F07417B1
:10431100900773F07418900774F0D2199000BDE003
:1043210090007BF09000DBE090007DF09000D9E000
:1043310090007CF0900090E090007EF0900109E008
:1043410090007FF09000F3E0B4011790002A740F01
:10435100F0A374FFF090002CE4F0A3F0740290003D
:10436100F3F09000F3E0B4034190002CE0FEA3E0F1
:10437100FF90002AE0FCA3E0FD126F627410126F3F
:10438100177408120039EF9000F2F0EF700674FF15
:104391009000F2F074009000F3F090002BE0900098
:1043A100A9F090002AE09000AAF0900084E090002B
:1043B10081F0900083E0900080F09000B2E0C3941F
:1043C1001E50569000B2E0F404241E900082F0903A
:1043D1000082E075F00684FF7E008F72900082E01B
:1043E10075F00684ADF07C008D73900080E0D3956C
:1043F10073400D900080E0C39573900080F0800FB2
:10440100900080E02406C39573900080F0057290BF
:104411000081E02572900081F0900081E0900048D9
:10442100F0900048E0241E900049F0900048E0D34D
:10443100943C400B900048E0C3943C900048F090BD
:104441000049E0D3943C400B900049E0C3943C9078
:104451000049F090004EE4F090004EE4F0900048E6
:10446100E0643B6007900048E0B43C20900048E0E5
:10447100B43B06740290004EF0900048E0B43C0654
:1044810090004E7401F09000487401F090004FE4E8
:10449100F0900049E0643B6007900049E0B43C20A3
:1044A100900049E0B43B06740290004FF09000493F
:1044B100E0B43C0690004F7401F09000497401F0A3
:1044C100900084E0FE9000E7E02E900052F0900012
:1044D10052E0641E6007900052E0B43C0690005226
:1044E100E004F0900052E0641D6007900052E0B4D7
:1044F1003B06900052E014F0900052E0D3943C400F
:104501000B900052E0C3943C900052F0900052E0B6
:10451100D3941E400D900052E0C3941E900053F0BE
:10452100800A900052E0241E900053F0755C1E90AA
:104531000084E0FE9000CAE0D39E5013900084E016
:10454100FE9000CAE0F4042E0490004AF08013901B
:104551000084E0243CFE9000CAE0F4042E049000A4
:104561004AF090004AE0B41E06741F90004AF09091
:10457100004AE0B41D06741C90004AF090004AE025
:10458100B43C0690004A7401F090004AE0B43B0646
:10459100743A90004AF090004AE0D3941E400D9086
:1045A100004AE0C3941E90004CF0800A90004AE05B
:1045B100241E90004CF090004AE090004BF09000D7
:1045C1004CE090004DF012019C22C293C294C29122
:1045D100C292C287C290E5B554EFF5B5E5B554DF97
:1045E100F5B5C296C295C2A0C297C2A2C2A1E5B555
:1045F10054BFF5B5E5B5547FF5B5E5B554FBF5B553
:10460100C208755D469000CDE07005756C028003AF
:10461100756C0375530075520090001274FFF0A37E
:1046210074DCF0C20FC21174C8900040F074C890DD
:104631000044F0755100755000C203754500E56EE8
:10464100B41303756E00756200900020E4F0A3F0CE
:10465100756F10C20BC20CC20DC20EC2027555009D
:10466100755400900014E4F0A3F0900016E4F0A358
:10467100F0C21D90001074FFF0A374DCF090000CE8
:1046810074FFF0A374DCF090000E74FFF0A374DCEF
:10469100F090000474FFF0A374DCF090000674FF46
:1046A100F0A374DCF075570075560090008FE0752B
:1046B100F032A4FFAEF0900028EEF0A3EFF0740208
:1046C1009008EDF022755900755800AE58AF597435
:1046D1001CC39F74019E50030247BA906BFE1200E7
:1046E10048E493645F6023906BFE120048E4936496
:1046F1007E6017906BFE120048E4936481600B901A
:104701006BFE120048E493B4840302479AAE58AF9B
:1047110059906BFE120048E493900083126F480F8A
:10472100BF00010EE0FC906BFE120048ECFEE4932A
:10473100FFEEC39F5026AE58AF590FBF00010E9038
:104741006BFE120048AE58AF59E493FC906BFE1219
:104751000048E493900083126F48ECF0AE58AF59D3
:10476100906BFE120048E493900083126F48E0FCC6
:10477100906C00120048ECFCE493FDECD39D4019D1
:10478100906C00120048E493FC906BFE120048E428
:1047910093900083126F48ECF0AE58AF5974022F1A
:1047A100FF50010E8E588F597859740126F6500426
:1047B10018E436F640030246CC22755900755800BC
:1047C100AE58AF597432BE00039F5003024888901F
:1047D1006D1B120048E493900083126F480FBF00D5
:1047E100010EE0FC906D1B120048ECFEE493FFEE1D
:1047F100C39F5026AE58AF590FBF00010E906D1BDD
:10480100120048AE58AF59E493FC906D1B1200485A
:10481100E493900083126F48ECF0AE58AF59906D5D
:104821001B120048E493900083126F48E0FC906DE6
:104831001D120048ECFCE493FDECD39D4019906DF2
:104841001D120048E493FC906D1B120048E4939004
:104851000083126F48ECF0AE58AF59742D6F4E7053
:1048610006755933755800AE58AF5974022FFF5071
:10487100010E8E588F597859740126F6500418E4A8
:1048810036F640030247C122755900755800AE58EB
:10489100AF597432BE00039F5003024956906D4ECA
:1048A100120048E493900083126F480FBF00010E7D
:1048B100E0FC906D4E120048ECFEE493FFEEC39FC6
:1048C1005026AE58AF590FBF00010E906D4E120029
:1048D10048AE58AF59E493FC906D4E120048E493F2
:1048E100900083126F48ECF0AE58AF59906D4E12A4
:1048F1000048E493900083126F48E0FC906D5012E1
:104901000048ECFCE493FDECD39D4019906D5012EE
:104911000048E493FC906D4E120048E493900083AC
:10492100126F48ECF0AE58AF59742D6F4E7006758A
:104931005933755800AE58AF5974022FFF50010E0C
:104941008E588F597859740126F6500418E436F6BA
:10495100400302488F2275A71085F97285FA737E8C
:10496100017F00E573126F17E5722FFF50010E8E64
:10497100588F59AC5AAD5BEF2DFDEE3CFC8C5A8D36
:104981005BD293D291E55BF5FBE55AF5FCE55BF56E
:10499100EBE55AF5EC75A7002275A71085F972852C
:1049A100FA737E017F00E573126F17E5722FFF50D6
:1049B100010E8E588F597E017F76900108E0126FAB
:1049C10017AC58AD59ED2FFFEC3EFE8E5A8F5BE5CB
:1049D1005BF5FDE55AF5FE900077E4F075A70074EC
:1049E10012900055F02285F97285FA737E017F00DD
:1049F100E573126F17E5722FFF50010E8E588F5914
:104A010090001AE0FCA3E0FDEF2DFDEE3CFC8C5A7A
:104A11008D5BE55BF5FDE55AF5FE22056322A2DC1F
:104A2100B34026A296B3B34012A295B3B3400CA2F1
:104A3100A0B3B34006A297B3B350067419900055C2
:104A4100F0C296C295C2A0C29775D8402285A771BF
:104A510075A710A2D8B3400AC2939000E9E0700292
:104A6100C294A2D9B34002C294A2DAB3400AC2915D
:104A71009000E9E07002C292A2DBB34002C292A2AE
:104A8100DCB340089000D7E0900077F075D84085FE
:104A910071A72290F800E4936406600280FE120080
:104AA1009E75A70075D80075D90475DE0975D840C3
:104AB10075A71075D80075D90475DA0975DB097504
:104AC100DC0975DD0975DE0975D84075A70012008E
:104AD100FB7509C875080012062475A70FE5FC903F
:104AE1000064F0E5FB900065F0E5FA900066F0E502
:104AF100F9900067F075A70090F800E493F526128D
:104B0100074390089AE0D39403500790089AE0B4C1
:104B11000106740090089AF090089AE09008F1F06C
:104B210074019000CCF090089AE090680EF8282863
:104B310073802A802875A70F75F30F75A700A2A3AC
:104B4100400674029000CCF0801375A70F75F3171F
:0D4B510075A700A2A4400674029000CCF0ED
:0C680E00024B32024B34024B36024B4B63
:104B5E009000CCE0B4022AC215120AEC7402900046
:104B6E00CCF090089AE090681AF82828738010808C
:0F4B7E000E74009000DBF0800674009000E8F0E9
:0C681A00024B7B024B7D024B7F024B8740
:104B8D008028D215120A0174019000CCF090089A79
:104B9D00E0906826F82828738010800E740090002D
:0A4BAD00DBF0800674009000E8F0D1
:0C682600024BA5024BA7024BA9024BB18C
:104BB70090F807E493900071F0900071E04408903A
:104BC7000071F0900071E054FE900071F01203BD87
:104BD700123F329008A7E090016FF09008A8E0908C
:104BE7000170F09008A9E0900171F090016FE070FA
:104BF7000C900170E07006900171E060028004C2C1
:104C07001A8002D21A9000BDE00490007BF0900158
:104C170027E0B4FF067400900127F0900128E0B464
:104C2700FF067400900128F01246C690F802E4933C
:104C3700B4050512488980031247BB74009000F33E
:104C4700F0124089E5B54401F5B57406900057F0B8
:104C57007400900058F07401900059F090F802E445
:104C67009390005AF090F803E49390005BF090F86B
:104C770004E49390005CF0740690005DF090005A95
:104C8700E0B40506740590005DF0743A90005EF09C
:104C9700740390005FF07407900060F07401900057
:104CA70061F090F805E493900062F090F806E493C1
:104CB700900063F0740090006BF0740090006CF04B
:104CC700740090006DF0740090006EF07400900016
:104CD7006FF07400900070F074FF900072F0A2B64D
:104CE700B39204A2B3B39205A2A4B39217A2A3B33B
:104CF7009218900073E4F0756E00743A900783F091
:104D070074FD900784F0900074E4F0756D019000D5
:104D170055E4F09000CDE0B40106741A900055F008
:104D2700C216756200C209D20AC202757000C219A2
:104D37001205C6755E00756A007560007564327588
:104D470065007566007567007568007569009000F5
:104D570020E4F0A3F0756B00D2B2D2A4D2B0D2B1E6
:104D6700D2A3D2A7D2A6D2A5D2B77E017F00900048
:104D7700AAE0126F179000A9E02FFF50010E9000D4
:104D87002AEEF0A3EFF0EFD394FFEE940F400790D5
:104D9700002AE4F0A3F09000F2E0700674FF9000A0
:104DA700F2F09000CDE07005756C028003756C031E
:104DB700740090010FF07400900112F0740A9001D2
:104DC70013F074299006C9F0742A9006CDF0740583
:104DD7009006D9F074069006DDF074079006E1F0AE
:104DE70074089006E5F0741B9006E9F0741C9006B1
:104DF700EDF07400900775F07400900776F074007A
:104E0700900777F07400900778F0740090077DF0B2
:104E1700740090077EF0740090077FF0740090078D
:104E270080F0D29CE56FD394104003756F10900605
:104E3700CAE0D3940C400674009006CAF09006CEE0
:104E4700E0D3940C400674009006CEF09006D2E0B2
:104E5700D3940C400674009006D2F09006D6E0D3A7
:104E6700940C400674009006D6F09006DAE0D394CE
:104E77000C400674009006DAF09006DEE0D3940C3E
:104E8700400674009006DEF09006E2E0D3940C40F2
:104E97000674009006E2F09006E6E0D3940C400614
:104EA70074009006E6F09006EAE0D3940C4006748E
:104EB700009006EAF09006EEE0D3940C40067400EA
:104EC7009006EEF0D2EC75CF01A298B34005C298D8
:104ED700120C54E54C6006A299B3B340028005C298
:104EE700991210E0E54D64016005E54DB4040280B8
:104EF700D5C28E7E107F00E563126F17E58D75F0C2
:104F070010A4FDACF0EF2DFDEE3CFCE58B75F01029
:104F170084FF7E00ED2FFFEC3EFE8E528F53D28E24
:104F27009000B0E060099000B0E0C3943D4002807B
:104F370056900022126F25900022E0FEA3E0FF901A
:104F47000024E0FCA3E0FDEFB5053CEEB50438B264
:104F570013A203B34013A213B34008E5B54404F505
:104F6700B58006E5B554FBF5B5900024E0FEA3E057
:104F7700FF900026E0FCA3E0FDEF2DFDEE3CFC904A
:104F87000024ECF0A3EDF09000BDE060099000BDB7
:104F9700E0C394034002806F123027A203400890B9
:104FA70000A7E0F544801BE55EC3955F5005754497
:104FB70000800F900094E0C3956050069000BAE01F
:104FC700F544E54475F002A4FFAEF090088FEEF0CB
:104FD700A3EFF0AC2DAD2EEDD39FEC9E4004C2A104
:104FE700800B900073E0C394485002D2A19000BD9B
:104FF700E0B40213A2A1B34008E5B554BFF5B580EC
:1050070006E5B54440F5B59000BDE0B4031C123188
:1050170042AE2DAF2E90088FE0FCA3E0FDEFD39DAD
:10502700EE9C4004D2A18002C2A1A2B6300401B313
:1050370050030255FCA2B6300401B350030255FCDD
:10504700A2B6300601B35003025534756D00055DF5
:10505700A208B3B35013AE52AF53900012E0FCA3B3
:10506700E0FDEDC39FEC9E400302518AE56CB4035B
:105077002EA21DB34022E55DB43B03756C01E55DCF
:10508700C3943B50069000557401F0E55DD3943B03
:1050970040067402900055F0755D01D21D805EE5F3
:1050A7006CB40206756C01755D3BE55DB43B057537
:1050B7005D018049900055E07034E55DC3943B5035
:1050C700069000557401F0E55DD3943B40067402E9
:1050D700900055F0E55DC3943B5002D216E55DD3D1
:1050E700943B4002D216C296C295C2A0C2979000C6
:1050F700CDE0B401051245CB8003755D01AE54AF19
:1051070055AC52AD53EF2DFDEE3CFC74028C068D71
:10511700071200398E548F559000B0E06009900057
:10512700B0E0C3943D40028043900022E0FEA3E03C
:10513700FF9000B0E08E048F05FF126F0774018C9B
:10514700068D07120039900026EEF0A3EFF09000CD
:1051570026E0F8A3E0900024C8F0A3C8F09000224E
:10516700E4F0A3F0C213E5B554FBF5B5A2A4B34030
:1051770002C217A2A3B34002C218A216B34002C2CA
:1051870016803AAE54AF55AC52AD53EF2DFDEE3C01
:10519700FC74018C068D071200398E548F55E56C0F
:1051A700C39402500DAC52AD5374B8C39D740B9C9D
:1051B700400280091245CB7406900055F0E55DB4B6
:1051C7003B127403900055F0D2169000CDE0B40165
:1051D700031245CBAE56AF57AC52AD53EF2DFDEE94
:1051E7003CFC8C568D57AE52AF53EFD39DEE9C408F
:1051F70011900018E0FAA3E0FBEBC394E8EA9403EC
:1052070040028006900018126F25900016E0FEA35A
:10521700E0FFAC52AD53EF2DFDEE3CFC900016ECD9
:10522700F0A3EDF09000CDE0B40118AE52AF537487
:1052370005126F177401120039900012EEF0A3EFF8
:10524700F08011AE52AF537402126F17900012EE36
:10525700F0A3EFF0900004E0FEA3E0FF74E8D39F13
:1052670074FD9E401FAC52AD53EFD39DEE9C400D95
:10527700126F62900004EEF0A3EFF0800790000435
:10528700E4F0A3F090000CE0FEA3E0FF74E8D39FE6
:1052970074FD9E401FAC52AD53EFD39DEE9C400D65
:1052A700126F6290000CEEF0A3EFF0800790000CF5
:1052B700E4F0A3F0900006E0FEA3E0FF74E8D39FBC
:1052C70074FD9E401FAC52AD53EFD39DEE9C400D35
:1052D700126F62900006EEF0A3EFF08007900006D1
:1052E700E4F0A3F090000EE0FEA3E0FF74E8D39F84
:1052F70074FD9E401FAC52AD53EFD39DEE9C400D05
:10530700126F6290000EEEF0A3EFF0800790000E90
:10531700E4F0A3F0C28E758D00758B007563007580
:105327005301755200D28EE55D240E75F00F84AFE0
:10533700F07E00EF4E60030253C3E56C6013AE547A
:10534700AF55740F126F17900014EEF0A3EFF080B3
:105357000F900016E0F8A3E0900014C8F0A3C8F07F
:10536700900014E0FEA3E0FFEF4E600B7C797DA96F
:10537700126E058E508F51900016E4F0A3F0AE50D8
:10538700AF517428BE00039F5010E5622FFF5001F4
:105397000E74011200398E508F518551629000D4DE
:1053A700E0A850B8000DD395514008E5519000543E
:1053B700F080099000D4E014900054F0E55D640B90
:1053C7006005E55DB429099000BDE06003122CDD9E
:1053D700900052E0655D6007900053E0B55D03758E
:1053E7006E00A209B35006A208B3B3400302549C4F
:1053F700900089E0B4017390010BE0B4021412121B
:1054070081900078E075F0BCA4FFAEF08E5A8F5BF8
:105417008056E56675F00A84FF7E009005831200CA
:1054270048E0F559755800AE58AF599000AEE012F4
:105437006F1774648E048F05FF126F078C5A8D5B8C
:10544700E55B900050F0AE58AF59900087E0126FBF
:105457001774648E048F05FF126F0774BC8C068D5A
:1054670007126F178E5A8F5B8017900087E075F0D1
:10547700BCA4FFAEF08E5A8F5B9000AEE090005058
:10548700F0E560C394CC5006E55B455A7002800393
:10549700124957D209E56CB40106E55D6411600253
:1054A7008009756F009000567401F0E56C70799073
:1054B70000D0E0600D900077E0A850B80006955145
:1054C700400280389000D0E0B40217900048E065B1
:1054D7005D6007900049E0B55D03756F03756B006C
:1054E700800CC200756B00900020E4F0A3F09000E0
:1054F70077E060067409900055F0802C900048E032
:10550700655D6007900049E0B55D1D756F0090000F
:1055170048E0B55D069000567401F0900049E0B58B
:105527005D067402900056F0A206B39204A206B379
:1055370030B601B350030255FC756D01E5B5440162
:10554700F5B57430900073F0A2069204E55DD3942C
:105557004A4014D208E55DD39485400B740490004B
:1055670055F0D216755D469000D8E0B40107E5699D
:10557700C3944140028018E569C39414500874131A
:10558700900055F08006740E900055F01245CB90B0
:10559700005DE0FE90005AE0C39E400990005AE08B
:1055A700D39408400974FB900055F01245CB900046
:1055B7005BE0601590005BE0FE900059E06E6009CB
:1055C70074FC900055F01245CB90005CE06015909C
:1055D700005CE0FE90005EE06E600974FE9000558E
:1055E700F01245CB90089AE06006900108E060024F
:1055F7008003120BD7A216B34008C296C295C2A069
:10560700C297900108E0600CAE50AF517414BE0011
:10561700059F40028037900090E0906832F8282874
:1056270073802A8028A2A3B35005A218B340028032
:105637000512499AD2188015A2A4B35005A217B330
:0D5647004002800512499AD21780028000AF
:1068320002562802562A02562C02563F025652028D
:026842005654AA
:10565400A20BB3B3500890004AE0655D60030257A3
:105664001FA201B35006A200B3B3400302571B129A
:105674003D7590011CE0601F90001EE0FEA3E0FF5A
:10568400900114E0126F1774C88E048F05FF126F17
:10569400078C5A8D5B800A90001EE0F55AA3E0F552
:1056A4005B9000B4E0B40123AE5AAF5B745E126F3A
:1056B4001774058E048F05FF126F07AE58AF59EDAE
:1056C4002FFFEC3EFE8E5A8F5B8021AE5AAF5B7487
:1056D4005E126F17740A8E048F05FF126F07AE589F
:1056E400AF59ED2FFFEC3EFE8E5A8F5BAE5AAF5B87
:1056F40090003EE0FCA3E0FDEF2DFDEE3CFC8C5A57
:105704008D5BE55BF5FBE55AF5FCD2939000E9E08F
:105714007002D29475A700C20BD20DA20CB3B35081
:105724000890004BE0655D6003025898A201B350F5
:1057340006A200B3B34003025894123D75A202B30B
:1057440050030257E690011CE0D39401401F9000DF
:105754001EE0FEA3E0FF900115E0126F1774C88EDF
:10576400048F05FF126F078C5A8D5B800A90001E10
:10577400E0F55AA3E0F55B9000B4E0B40123AE5A1F
:10578400AF5B745E126F1774058E048F05FF126F82
:1057940007AE58AF59ED2FFFEC3EFE8E5A8F5B805B
:1057A40021AE5AAF5B745E126F17740A8E048F05B4
:1057B400FF126F07AE58AF59ED2FFFEC3EFE8E5A25
:1057C4008F5BAE5AAF5B90003EE0FCA3E0FDEF2D93
:1057D400FDEE3CFC8C5A8D5BE55BF5E9E55AF5EA98
:1057E400D2949000E9E0B4020CAE50AF517405BEFF
:1057F40000069F400302589190011CE0D39401409D
:105804001BAE2BAF2C900115E0126F1774C88E04D9
:105814008F05FF126F078C5A8D5B8006852B5A8586
:105824002C5B9000B4E0B40123AE5AAF5B745E12FB
:105834006F1774058E048F05FF126F07AE58AF59AA
:10584400ED2FFFEC3EFE8E5A8F5B8021AE5AAF5B8C
:10585400745E126F17740A8E048F05FF126F07AE01
:1058640058AF59ED2FFFEC3EFE8E5A8F5BAE5AAF08
:105874005B90003EE0FCA3E0FDEF2DFDEE3CFC8CD4
:105884005A8D5BE55BF5E9E55AF5EAD29475A70014
:10589400C20CD20EA20DB3B3500890004CE0655D6B
:1058A4006003025966A201B35006A200B3B34003D9
:1058B400025962123D7590011CE0D39402401F907E
:1058C400001EE0FEA3E0FF900116E0126F1774C8FB
:1058D4008E048F05FF126F078C5A8D5B800A90002F
:1058E4001EE0F55AA3E0F55B9000B4E0B40123AEEA
:1058F4005AAF5B745E126F1774058E048F05FF1226
:105904006F07AE58AF59ED2FFFEC3EFE8E5A8F5BFA
:105914008021AE5AAF5B745E126F17740A8E048FC7
:1059240005FF126F07AE58AF59ED2FFFEC3EFE8E08
:105934005A8F5BAE5AAF5B90003EE0FCA3E0FDEFF4
:105944002DFDEE3CFC8C5A8D5BE55BF5EBE55AF5E1
:10595400ECD2919000E9E07002D29275A700D20BCC
:10596400C20DA20EB3B3500890004DE0655D600314
:10597400025ADFA201B35006A200B3B34003025A95
:10598400DB123D75A202B35003025A2D90011CE0B4
:10599400D39401401F90001EE0FEA3E0FF90011786
:1059A400E0126F1774C88E048F05FF126F078C5AAC
:1059B4008D5B800A90001EE0F55AA3E0F55B900031
:1059C400B4E0B40123AE5AAF5B745E126F17740572
:1059D4008E048F05FF126F07AE58AF59ED2FFFEC01
:1059E4003EFE8E5A8F5B8021AE5AAF5B745E126F9F
:1059F40017740A8E048F05FF126F07AE58AF59ED66
:105A04002FFFEC3EFE8E5A8F5BAE5AAF5B90003E8A
:105A1400E0FCA3E0FDEF2DFDEE3CFC8C5A8D5BE534
:105A24005BF5EDE55AF5EED2929000E9E0B4020C94
:105A3400AE50AF517405BE00069F4003025AD89081
:105A4400011CE0D39403401BAE2BAF2C900117E054
:105A5400126F1774C88E048F05FF126F078C5A8D4E
:105A64005B8006852B5A852C5B9000B4E0B401233F
:105A7400AE5AAF5B745E126F1774058E048F05FF08
:105A8400126F07AE58AF59ED2FFFEC3EFE8E5A8FC2
:105A94005B8021AE5AAF5B745E126F17740A8E047A
:105AA4008F05FF126F07AE58AF59ED2FFFEC3EFE86
:105AB4008E5A8F5BAE5AAF5B90003EE0FCA3E0FDD4
:105AC400EF2DFDEE3CFC8C5A8D5BE55BF5EDE55A64
:105AD400F5EED29275A700D20CC20EE56F90684421
:085AE400F82828739000F0E09F
:03684400025AE80D
:105AEC00906877F828287312260C801212260C80E6
:0E5AFC000D12269680081227428003122742C0
:0F687700025AF3025AF8025AFD025B02025B0753
:105B0A00756F010260EA12286E122985756F02020A
:105B1A0060EAA203B340139000D5E075F01DA4FF1C
:105B2A00AEF090001AEEF0A3EFF0122D21122C1312
:105B3A009000D9E0B404028003025C0B900883E071
:105B4A00FEA3E0FF740A126F17900014E0FCA3E0B2
:105B5A00FD74098F02FF126F078D078C038E048A6A
:105B6A00058B06126E05900887EEF0A3EFF074F02D
:105B7A00BE00039F500B74F0900887F8E4F0E8A386
:105B8A00F0E5357003753501900887E0FEA3E0FF64
:105B9A00E5352FFF50010E900887EEF0A3EFF09045
:105BAA000014E0FCA3E0FD7478D39D74059C401FAB
:105BBA009008E8E08C068D07126F17745A8E048FCE
:105BCA0005FF126F07900010ECF0A3EDF0802F9004
:105BDA000014E0FEA3E0FF74098E048F05FF126F24
:105BEA00079008E8E08C068D07126F17740A8E0476
:105BFA008F05FF126F07900010ECF0A3EDF0025C26
:105C0A00D99000D9E0B402028003025CD9900883DB
:105C1A00E0FEA3E0FF740A126F17900014E0FCA3E1
:105C2A00E0FD74098F02FF126F078D078C038E0443
:105C3A008A058B06126E05900887EEF0A3EFF074C2
:105C4A0078BE00039F500B7478900887F8E4F0E858
:105C5A00A3F0E5357003753501900887E0FEA3E0EF
:105C6A00FFE5352FFF50010E900887EEF0A3EFF005
:105C7A00900014E0FCA3E0FD7478D39D74059C4069
:105C8A001F9008E8E08C068D07126F17745A8E046D
:105C9A008F05FF126F07900010ECF0A3EDF0802F34
:105CAA00900014E0FEA3E0FF74098E048F05FF1232
:105CBA006F079008E8E08C068D07126F17740A8E3A
:105CCA00048F05FF126F07900010ECF0A3EDF0753A
:0A5CDA006F03A2244015900056E06D
:06684700025B10025B1C65
:105CE400906886F82828738008756F0A8003756F9A
:015CF4000BA4
:09688600025CEB025CED025CF225
:105CF5000260EA9006CAE06006750801122E4FA2FE
:105D050026B3B35008900781E0640760028009E577
:105D1500B54410F5B5025DBE9000BEE0D3940240D7
:105D250045900092E02403A850B80004955150090D
:105D3500900094E0D395605002800ED201A21C40E1
:105D4500067408900055F0D21C900092E0A850B857
:105D55000005D39551500B900094E02403C3956042
:105D65005002C2018053900092E02403A850B8006D
:105D75000495515010E55EC3955F5009900094E07D
:105D8500D395605002800ED201A21C400674089083
:105D95000055F0D21C900092E0A850B80005D395AC
:105DA500515014E55F240FC3955E400B900094E0BD
:105DB5002403C395605002C201A2014002C21CA285
:105DC50026B3500DA201B35008900781E064076027
:105DD500028006E5B554EFF5B59000D8E07007E50B
:105DE50069C3941440028002D2019000CDE0B40151
:105DF50002D201A2014005756F04800A756F1090EB
:0D5E05000020E4F0A3F00260EA9000BEE08F
:06684D00025CF8025E0E81
:105E120090688FF8282873121397801212139780B4
:0E5E22000D12154A8008121601800312160197
:0F688F00025E19025E1E025E23025E28025E2D6B
:105E30009006CEE06006750802122E4F756F059031
:105E4000010BE0B40205A203B340028012121281DA
:105E5000900078E0F528752700752A6475290002FE
:105E600060EA12175A756F069006D2E06006750850
:105E700003122E4F9006D6E06006750804122E4FCE
:105E80000260EA900050E06006A203B3B3400280D3
:105E90000DE55DD3941E5006900050E014F01219E9
:105EA000E3756F079006DAE06006750805122E4F5D
:105EB0009006DEE06006750806122E4F0260EA903A
:105EC000010BE0B40203121308121E4B756F089009
:105ED00006E2E06006750807122E4F9006E6E060C5
:105EE00006750808122E4F0260EA121F2D756F0901
:105EF0000260EA1223059000CAE0700D123D9390F3
:105F000000E9E0B40203123E12A20BB35005A20D49
:105F1000B340028008D20BD20CD20DD20E756F1096
:105F20009006EAE06006750809122E4F9006EEE032
:105F3000600675080A122E4F0260EA900042E0C324
:105F400094465022C2967446900042F0900010E0B1
:105F5000FEA3E0FFAC52AD53EF2DFDEE3CFC9000F4
:105F60000CECF0A3EDF090004EE0B4011DE53524FB
:105F700006F535900887E0FEA3E0FF74062FFF507A
:105F8000010E900887EEF0A3EFF090004EE0B4020F
:105F90001DE535240CF535900887E0FEA3E0FF747D
:105FA0000C2FFF50010E900887EEF0A3EFF085351F
:105FB00059755800900048E0F572123FF2E55B9089
:105FC0000042F0900008E558F0A3E559F0E5729022
:105FD0000043F0C210900887E0F558A3E0F559900F
:105FE0000048E0F572123FF2E55B900040F090004F
:105FF00000E558F0A3E559F0E572900041F0C20FBA
:10600000E56CB40105756F0B8003756F030260EAE0
:10601000900046E0C394465022C2A07446900046C9
:10602000F0900010E0FEA3E0FFAC52AD53EF2DFD69
:10603000EE3CFC90000EECF0A3EDF090004FE0B4CD
:10604000011DE5352406F535900887E0FEA3E0FF45
:1060500074062FFF50010E900887EEF0A3EFF0902A
:10606000004FE0B4021DE535240CF535900887E0BB
:10607000FEA3E0FF740C2FFF50010E900887EEF096
:10608000A3EFF0853559755800900049E0F572127C
:106090003FF2E55B900046F090000AE558F0A3E57A
:1060A00059F0E572900047F0C212900887E0F55869
:1060B000A3E0F559900049E0F572123FF2E55B90DC
:1060C0000044F0900002E558F0A3E559F0E5729025
:1060D0000045F0C211E56CB40103756C00756F03E7
:0A60E0008008800680048002800022
:10685300025E62025E83025EBF025EEA025EF302D2
:106863005F3B0260100260E20260E40260E60260E5
:04687300E80260EAED
:1060EA00900040E0B55D0280030261A6A20F4072F3
:1060FA00900000E0FEA3E0FFEF4E6021AE54AF55E2
:10610A00900000E0FCA3E0FD12000374068E048FE9
:10611A0005FF126F07900000ECF0A3EDF09000412C
:10612A00E0601A900000E0FEA3E0FFAC54AD55EF2A
:10613A002DFDEE3CFC900000ECF0A3EDF090004148
:10614A00E0D39401401A900000E0FEA3E0FFAC54B3
:10615A00AD55EF2DFDEE3CFC900000ECF0A3EDF008
:10616A00D20FAE52AF53900000E0FCA3E0FDEFC3A4
:10617A009DEE9C40271249E7D296C20F74C8900040
:10618A0040F0900010E0FEA3E0FFAC52AD53EF2DBB
:10619A00FDEE3CFC900004ECF0A3EDF0A20FB3B3CB
:1061AA005007900040E0B55D0280271249E7D29679
:1061BA0074C8900040F0C20F900010E0FEA3E0FF08
:1061CA00AC52AD53EF2DFDEE3CFC900004ECF0A375
:1061DA00EDF0900042E0B55D028003026291A210E8
:1061EA004072900008E0FEA3E0FFEF4E6021AE543B
:1061FA00AF55900008E0FCA3E0FD12000374068E80
:10620A00048F05FF126F07900008ECF0A3EDF090E1
:10621A000043E0601A900008E0FEA3E0FFAC54AD32
:10622A0055EF2DFDEE3CFC900008ECF0A3EDF0904C
:10623A000043E0D39401401A900008E0FEA3E0FF77
:10624A00AC54AD55EF2DFDEE3CFC900008ECF0A3EC
:10625A00EDF0D210AE52AF53900008E0FCA3E0FD7F
:10626A00EFC39DEE9C4020C2967446900042F0C255
:10627A0010900010E0FAA3E0FBEB2FFFEA3EFE903D
:10628A00000CEEF0A3EFF0A210B3B3500790004257
:10629A00E0B55D028024C2967446900042F0C210B6
:1062AA00900010E0FEA3E0FFAC52AD53EF2DFDEEDF
:1062BA003CFC90000CECF0A3EDF0AE52AF53900012
:1062CA0004E0FCA3E0FDEFC39DEE9C400F1249E7FA
:1062DA00D29590000474FFF0A374DCF0AE52AF5371
:1062EA0090000CE0FCA3E0FDEFC39DEE9C400CC2C5
:1062FA009590000C74FFF0A374DCF0900044E0B5B4
:10630A005D0280030263C1A2114072900002E0FEA6
:10631A00A3E0FFEF4E6021AE54AF55900002E0FCBF
:10632A00A3E0FD12000374068E048F05FF126F07A7
:10633A00900002ECF0A3EDF0900045E0601A9000A6
:10634A0002E0FEA3E0FFAC54AD55EF2DFDEE3CFCA0
:10635A00900002ECF0A3EDF0900045E0D3940140E8
:10636A001A900002E0FEA3E0FFAC54AD55EF2DFDFC
:10637A00EE3CFC900002ECF0A3EDF0D211AE52AF6D
:10638A0053900002E0FCA3E0FDEFC39DEE9C402782
:10639A001249E7D2A0C21174C8900044F0900010CC
:1063AA00E0FEA3E0FFAC52AD53EF2DFDEE3CFC90B6
:1063BA000006ECF0A3EDF0A211B3B350079000442D
:1063CA00E0B55D0280271249E7D2A074C890004464
:1063DA00F0C211900010E0FEA3E0FFAC52AD53EF03
:1063EA002DFDEE3CFC900006ECF0A3EDF09000468B
:1063FA00E0B55D0280030264ACA212407290000A0A
:10640A00E0FEA3E0FFEF4E6021AE54AF5590000AC4
:10641A00E0FCA3E0FD12000374068E048F05FF1250
:10642A006F0790000AECF0A3EDF0900047E0601AC5
:10643A0090000AE0FEA3E0FFAC54AD55EF2DFDEE4F
:10644A003CFC90000AECF0A3EDF0900047E0D394F6
:10645A0001401A90000AE0FEA3E0FFAC54AD55EFEC
:10646A002DFDEE3CFC90000AECF0A3EDF0D212AE4A
:10647A0052AF5390000AE0FCA3E0FDEFC39DEE9CEF
:10648A004020C2A07446900046F0C212900010E06C
:10649A00FAA3E0FBEB2FFFEA3EFE90000EEEF0A31C
:1064AA00EFF0A212B3B35007900046E0B55D028048
:1064BA0024C2A07446900046F0C212900010E0FE7A
:1064CA00A3E0FFAC52AD53EF2DFDEE3CFC90000E65
:1064DA00ECF0A3EDF0AE52AF53900006E0FCA3E05F
:1064EA00FDEFC39DEE9C400F1249E7D2979000063C
:1064FA0074FFF0A374DCF0AE52AF5390000EE0FCD0
:10650A00A3E0FDEFC39DEE9C400CC29790000E7471
:10651A00FFF0A374DCF09000DBE0B4020280030217
:10652A00663C900075E0D395655064900075E0F480
:10653A00042565FE9000DEE08E00F5F0E884FF7E1B
:10654A00008F72EFC39410500CEF8572F0A4FDAC6B
:10655A00F08D7280037572FF900075E0D3957240DA
:10656A000B900075E0C39572F5708003757000900A
:10657A0000F9E0D3957040069000F9E0F5709000BC
:10658A00FAE0C3957050069000FAE0F570807190B9
:10659A000075E0C39565FE9000DEE08E00F5F0E838
:1065AA0084FF7E008F72EFC39410500CEF8572F057
:1065BA00A4FDACF08D7280037572FF85725975580F
:1065CA0000900075E02559FFAE5850010E8E588F85
:1065DA005974FFBE0009D39F400585597080037521
:1065EA0070FF9000F9E0D3957040069000F9E0F54D
:1065FA00709000FAE0C3957050069000FAE0F570CA
:10660A00A203B3B3500D900076E0FE9000E6E0D30B
:10661A009E5002800A7407900055F0C2A28013753A
:10662A00A710E5CDC395704004C2A28002D2A2751C
:10663A00A700E56EC39413501DE56E75F00284AF92
:10664A00F07E00EF4E70051232FC800AA2EDB340D4
:10665A0005C2ED1232FCAE52AF537410C39F7427B9
:10666A009E400C900074E0C3945A40030267EAA269
:10667A0008B340091245CB7406900055F0A20AB33C
:10668A00500EE560D394334007E560C394CC4002D2
:10669A00804190010BE0B40214121281900078E05C
:1066AA0075F05EA4FFAEF08E5A8F5B800F90008764
:1066BA00E075F05EA4FFAEF08E5A8F5BE55B455A3B
:1066CA006011E5B54401F5B57430900073F01249D4
:1066DA0057D20A900074E0D394014007E560C3944E
:1066EA001A40028002C20A9006CAE06006750801D2
:1066FA00122E4F9006CEE06006750802122E4F90B9
:10670A0006D2E06006750803122E4F9006D6E060A6
:10671A0006750804122E4F9006DAE0600675080521
:10672A00122E4F9006DEE06006750806122E4F9074
:10673A0006E2E06006750807122E4F9006E6E06052
:10674A0006750808122E4F9006EAE06006750809D9
:10675A00122E4F9006EEE0600675080A122E4F9030
:10676A000074E0C3945A5010E56EB4130990007493
:10677A00E004F0756E00803FE56EB41303756E0099
:10678A00C28E758D00758B00756300755301755245
:10679A0000D28E900073E0C394485008900073E0D2
:1067AA0004F080067448900073F0900073E0B448D7
:1067BA0006E5B554FEF5B5900074E0D394014007A0
:1067CA00E569C3944140028006740E900055F0902A
:1067DA00089AE06006900108E060028003120BD775
:0367EA00024ECD8F
:10689E000000010001400160018001A001C001E083
:1068AE0002000300039603B603D603F404000500AA
:1068BE000512052405360548055A056C057E05901A
:1068CE0005A805C005DE0600061406280646066E57
:1068DE0006AE05CF06EE00FF013F015F017F019F6F
:1068EE0001BF01DF01FF02FF039503B503D503F3DB
:1068FE0003FF04FF05110523053505470559056BF3
:10690E00057D058F05A705BF05CE05F106130627E4
:10691E000645066D06AD06ED05DD06FF0FAA0FA5B1
:10692E000F9F0F9A0F940F8D0F870F800F780F7197
:10693E000F680F600F570F4E0F450F3B0F300F258F
:10694E000F1A0F0E0F020EF50EE80EDB0ECC0EBE5A
:10695E000EAE0E9F0E8E0E7D0E6C0E5A0E470E3420
:10696E000E200E0C0DF70DE20DCB0DB50D9D0D8508
:10697E000D6D0D540D3A0D200D050CE90CCE0CB11C
:10698E000C940C760C580C3A0C1B0BFB0BDB0BBB54
:10699E000B9A0B790B570B350B130AF10ACE0AAB78
:1069AE000A870A640A400A1C09F809D409B0098C3E
:1069BE0009670943091F08FB08D608B2088E086A42
:1069CE000846082307FF07DC07B907960773075128
:1069DE00072F070D06EC06CA06AA068906690649A0
:1069EE00062A060A05EC05CD05B005920575055873
:1069FE00053C0520050504EA04CF04B5049C048279
:106A0E000469045104390422040B03F403DE03C8A1
:106A1E0003B2039D038903750361034D033B0328F2
:106A2E000316030402F202E102D102C002B002A078
:106A3E00029102820273026502570249023C022F42
:106A4E0002220216020901FD01F201E601DB01D06C
:106A5E0001C601BB01B101A7019D0194018B018209
:106A6E00017901700168016001580150014801412E
:106A7E0001390132012B0125011E01180111010BF3
:106A8E00010500FF00FA0FA60FA00F990F920F8BB2
:106A9E000F840F7C0F740F6B0F620F580F4E0F4346
:106AAE000F380F2C0F1F0F120F050EF70EE80ED812
:106ABE000EC80EB70EA50E930E800E6C0E580E421B
:106ACE000E2C0E150DFD0DE40DCB0DB10D950D79A2
:106ADE000D5D0D3F0D200D010CE10CC00C9E0C7CCC
:106AEE000C590C350C100BEA0BC40B9E0B760B4F8E
:106AFE000B260AFD0AD40AAA0A800A550A2A09FF99
:106B0E0009D409A8097C0950092508F908CD08A15E
:106B1E000875084A081E07F307C8079D077307493B
:106B2E00072006F706CE06A6067E06570630060A8C
:106B3E0005E405BF059B057705540532051004EFE6
:106B4E0004CE04AE048F047104530435041903FDFE
:106B5E0003E203C703AD0394037B0363034B0334C8
:106B6E00031E030802F302DE02CA02B602A302915A
:106B7E00027F026D025C024C023C022C021D020ED0
:106B8E00020001F201E401D701CA01BE01B101A662
:106B9E00019A018F0185017A01700166015D015331
:106BAE00014A014101390131012901210119011265
:106BBE00010B010400FD00F700F000EA00E400DE26
:106BCE0000D900D300CE00C900C400BF00BA00B582
:106BDE0000B100AD00A800A400A0009C0099009593
:106BEE000091008E008A008700840081007E007B69
:10009E0075B50075840175A70075FFA075EF069004
:1000AE000051E4F075C91075A70F75A1C775A700AB
:1000BE0075D90075CE0C75A70F75F1FE75F2FF752B
:1000CE00F30775F47875A4BA75A5FF75A60775AE16
:1000DE000075AFFF75D48175D5FF75D6FF75D7FF47
:1000EE0075A70075A20175A14775F8092275E60876
:1000FE0075E71075BC0175BE0475BD6C75BE0775D0
:10010E00BDA075BE0875BD0175BC0075BB1875BC6C
:10011E002075BA0875E88075D11375A70F75E105BE
:10012E0075E20075C7401245CB75970075978074C0
:10013E000A126EF77597C0E5975420700280F87515
:10014E008F0275A700D2AF75980075A90C75A70F11
:10015E0075AB4375ADFB75AC1E75A71075C91875DB
:10016E00CA0075CB0075C80475A700758912758E07
:10017E0004758C00758A00C2A9D28C758D00758BA2
:10018E0000D2ABD28E75B62075D944C2992290009A
:10019E0085E0900899F0900090E090089AF0900019
:1001AE0091E090089BF09000B0E090089CF09000D9
:1001BE00BDE090089DF09000CBE090089EF090007E
:1001CE00D9E090089FF09000DBE09008A0F090003E
:1001DE00E9E09008A1F09000F6E09008A2F09000FF
:1001EE00F7E09008A3F0900109E09008A4F09001C8
:1001FE0021E09008A6F090016FE09008A7F0900122
:10020E0070E09008A8F0900171E09008A9F09001BC
:10021E0008E09008AAF09000F2E09008ABF0900091
:10022E00A9E09008ACF09000AAE09008ADF0900024
:10023E00A4E09008AEF09000A5E09008AFF0900119
:10024E000EE09008B0F090010FE09008B1F0900130
:10025E0010E09008B2F0900111E09008B3F0900118
:10026E0012E09008B4F09006C9E09008B5F0900640
:10027E00CDE09008B6F09006D1E09008B7F0900669
:10028E00D5E09008B8F09006D9E09008B9F0900645
:10029E00DDE09008BAF09006E1E09008BBF0900621
:1002AE00E5E09008BCF09006E9E09008BDF09006FD
:1002BE00EDE09008BEF0900771E09008BFF0900757
:1002CE0072E09008C0F0900773E09008C1F09007BC
:1002DE0074E09008C2F0900775E09008C3F09007A4
:1002EE0076E09008C4F0900777E09008C5F090078C
:1002FE0078E09008C6F0900779E09008C7F0900774
:10030E007AE09008C8F090077BE09008C9F090075B
:10031E007CE09008CAF090077DE09008CBF0900743
:10032E007EE09008CCF090077FE09008CDF090072B
:10033E0080E09008CEF0900781E09008CFF0900119
:10034E0013E09008D0F0900114E09008D1F09001E5
:10035E0015E09008D2F0900116E09008D3F09001CD
:10036E0017E09008D4F0900118E09008D5F09001B5
:10037E0019E09008D6F090011AE09008D7F090019D
:10038E001BE09008D8F090011CE09008D9F0900086
:10039E00B7E09008DAF09000EFE09008DBF0900103
:1003AE0027E09008DCF0900128E09008DDF0229024
:1003BE000899E0900085F090089AE0900090F090F7
:1003CE00089BE0900091F090089CE09000B0F090B7
:1003DE00089DE09000BDF090089EE09000CBF0905C
:1003EE00089FE09000D9F09008A0E09000DBF0901C
:1003FE0008A1E09000E9F09008A2E09000F6F090DD
:10040E0008A3E09000F7F09008A4E0900109F090A6
:10041E0008A6E0900121F09008AAE0900108F09063
:10042E0008ABE09000F2F09008ACE09000A9F090DC
:10043E0008ADE09000AAF09008AEE09000A4F09015
:10044E0008AFE09000A5F09008B0E090010EF0909B
:10045E0008B1E090010FF09008B2E0900110F0901A
:10046E0008B3E0900111F09008B4E0900112F09002
:10047E0008B5E09006C9F09008B6E09006CDF09071
:10048E0008B7E09006D1F09008B8E09006D5F0904D
:10049E0008B9E09006D9F09008BAE09006DDF09029
:1004AE0008BBE09006E1F09008BCE09006E5F09005
:1004BE0008BDE09006E9F09008BEE09006EDF090E1
:1004CE0008BFE0900771F09008C0E0900772F090BE
:1004DE0008C1E0900773F09008C2E0900774F090A6
:1004EE0008C3E0900775F09008C4E0900776F0908E
:1004FE0008C5E0900777F09008C6E0900778F09076
:10050E0008C7E0900779F09008C8E090077AF0905D
:10051E0008C9E090077BF09008CAE090077CF09045
:10052E0008CBE090077DF09008CCE090077EF0902D
:10053E0008CDE090077FF09008CEE0900780F09015
:10054E0008CFE0900781F09008D0E0900113F09072
:10055E0008D1E0900114F09008D2E0900115F090CF
:10056E0008D3E0900116F09008D4E0900117F090B7
:10057E0008D5E0900118F09008D6E0900119F0909F
:10058E0008D7E090011AF09008D8E090011BF09087
:10059E0008D9E090011CF09008DAE09000B7F090D6
:1005AE0008DBE09000EFF09008DCE0900127F0907F
:1005BE0008DDE0900128F022754600900891E4F0E5
:1005CE00A3F0753000752F00754C00754D00C220DC
:1005DE00D22190089AE06002D21974FE900893F826
:1005EE00E4F0E8A3F074FE900897F8E4F0E8A3F0C6
:1005FE0074FE900895F8E4F0E8A3F0745A9008EBB6
:10060E00F0745A9008ECF0D222C21EC224C223C249
:10061E001FC226C22C22750B00750A00AE0AAF0B44
:10062E00AC08AD09EDC39FEC9E401674FF126EF739
:10063E0075CF01780B740126F6500418E436F65087
:10064E00DB22C2AF75D904758F0375B7A575B7F1E7
:10065E0090F800E4F0758F0175B7A575B7F1E52632
:10066E0090F800F075B7A575B7F190F801E4F07544
:10067E00B7A575B7F19008DFE090F802F075B7A551
:10068E0075B7F19008E3E090F803F075B7A575B76C
:10069E00F19008E0E090F804F075B7A575B7F19009
:1006AE0008E1E090F805F075B7A575B7F19008E28E
:1006BE00E090F806F075B7A575B7F19008E4E090F4
:1006CE00F807F0758F0075D944D2AF22900051E033
:1006DE00B4AB61C2AF75D90475B62275F522758FAC
:1006EE000375B7A575B7F1740090F600F0758F011C
:1006FE00755900755800AE58AF597445BE00279F06
:10070E00402475B7A575B7F1900899120048E0FC22
:10071E0090F600120048ECF07859740126F6500459
:10072E0018E436F650D0758F0075F51175B6207534
:10073E00D944D2AF22C2AF75F52275D904755900CE
:10074E00755800AE58AF597445BE00229F401F9099
:10075E00F600120048E493FC900899120048ECF061
:10076E007859740126F6500418E436F650D575D92A
:10077E004475F511D2AF22900051E0B4AA02800365
:10078E000208C2C2AF75D90475B62275F522758FEF
:10079E000375B7A575B7F1740090F400F075B7A5A1
:1007AE0075B7F1740090F200F075B7A575B7F174D6
:1007BE000090F000F075B7A575B7F1740090EE00DB
:1007CE00F0758F01755900755800AE58AF5974FF0A
:1007DE00C39F74019E402475B7A575B7F190008331
:1007EE00120048E0FC90F400120048ECF0785974C6
:1007FE000126F6500418E436F650CF755900755898
:10080E0000AE58AF5974FFC39F74019E402475B754
:10081E00A575B7F1900283120048E0FC90F2001229
:10082E000048ECF07859740126F6500418E436F6B8
:10083E0050CF755900755800AE58AF5974FFC39F0D
:10084E0074019E402475B7A575B7F190048312000C
:10085E0048E0FC90F000120048ECF0785974012644
:10086E00F6500418E436F650CF755900755800AEA0
:10087E0058AF5974FFC39F74019E402475B7A57578
:10088E00B7F1900683120048E0FC90EE001200488B
:10089E00ECF07859740126F6500418E436F650CF71
:1008AE00758F0075F51175B62075D944D2AF743AAF
:1008BE00900783F022900051E0B4AA028003020A4E
:1008CE0000C2AF75D90475B62275F522758F037502
:1008DE00B7A575B7F1740090EC00F075B7A575B7B4
:1008EE00F1740090EA00F075B7A575B7F174009039
:1008FE00E800F075B7A575B7F1740090E600F075D5
:10090E008F01755900755800AE58AF5974FFC39FCB
:10091E0074019E402475B7A575B7F190008312003F
:10092E0048E0FC90EC00120048ECF0785974012677
:10093E00F6500418E436F650CF755900755800AECF
:10094E0058AF5974FFC39F74019E402475B7A575A7
:10095E00B7F1900283120048E0FC90EA00120048C2
:10096E00ECF07859740126F6500418E436F650CFA0
:10097E00755900755800AE58AF5974FFC39F740176
:10098E009E402475B7A575B7F1900483120048E018
:10099E00FC90E800120048ECF07859740126F650ED
:1009AE000418E436F650CF755900755800AE58AF9E
:1009BE005974FFC39F74019E402475B7A575B7F196
:1009CE00900683120048E0FC90E600120048ECF01E
:1009DE007859740126F6500418E436F650CF758F08
:1009EE000075F51175B62075D944D2AF743A9007DB
:1009FE0083F022C2AF75D90475F52275590075586A
:100A0E0000AE58AF5974FFC39F74019E401F90F4FF
:100A1E0000120048E493FC900083120048ECF0783A
:100A2E0059740126F6500418E436F650D475590060
:100A3E00755800AE58AF5974FFC39F74019E401F86
:100A4E0090F200120048E493FC900283120048ECEE
:100A5E00F07859740126F6500418E436F650D47521
:100A6E005900755800AE58AF5974FFC39F74019E5C
:100A7E00401F90F000120048E493FC900483120093
:100A8E0048ECF07859740126F6500418E436F65006
:100A9E00D4755900755800AE58AF5974FFC39F7482
:100AAE00019E401F90EE00120048E493FC900683D6
:100ABE00120048ECF07859740126F6500418E4360A
:100ACE00F650D475F51175D944D2AF74019000CC9F
:100ADE00F0743A900783F09008F27401F022C2AFDE
:100AEE0075D90475F522755900755800AE58AF5971
:100AFE0074FFC39F74019E401F90EC00120048E4E7
:100B0E0093FC900083120048ECF07859740126F69D
:100B1E00500418E436F650D4755900755800AE5886
:100B2E00AF5974FFC39F74019E401F90EA001200DC
:100B3E0048E493FC900283120048ECF0785974015B
:100B4E0026F6500418E436F650D475590075580040
:100B5E00AE58AF5974FFC39F74019E401F90E800BA
:100B6E00120048E493FC900483120048ECF078598C
:100B7E00740126F6500418E436F650D475590075F3
:100B8E005800AE58AF5974FFC39F74019E401F901A
:100B9E00E600120048E493FC900683120048ECF045
:100BAE007859740126F6500418E436F650D475F5CB
:100BBE001175D944D2AF74029000CCF0743A9007FC
:100BCE0083F074029008F2F02274019000CCF09041
:100BDE00089AE0903CBBF828287380188016A2A3D0
:100BEE00400674029000CCF0800AA2A44006740263
:040BFE009000CCF0A7
:0C3CBB00020BE8020BEA020BEC020BF813
:100C02009000CCE0B40105A22AB34002801AD22A95
:100C12001245CB120A0174019000CCF01203BD12EE
:100C22003F32741B900055F09000CCE0B40206A253
:100C32002AB3B34002801AC22A1245CB120AEC74BC
:100C4200029000CCF01203BD123F32741B9000558B
:100C5200F022E54D64046006E59964FF600280318C
:100C6200A2204004D2208027E54D600874E6254D7D
:100C7200900055F0E54C600874F0254C900055F05A
:100C8200E54DB4010280FE754D00754C00C2208016
:100C920002C220E54D903CC7F8282873754D00E547
:100CA20099B4FF03754C01E599B4FE03754C02E556
:100CB20099B4FD03754C03E599B4FC03754C04E546
:100CC20099B4FA03754C05E599B4FB06754D01120A
:100CD20045CBE599B4F906754D041245CBE599B4B7
:100CE200F7331245CBC29C74AB900051F01206DA76
:100CF20074AA900051F09008F2E0B4010512078541
:100D020080031208C3900051E4F0D29C754D007527
:100D12004C007599F7E599D394E54007E599C3949A
:100D2200F04002801685994E754D027E017F00E5E6
:100D32004EC394E6126F178E318F32900891E4F011
:100D4200A3F0E599D394C24007E599C394E6400223
:100D5200802885994E754D0374E5C3954EF532751D
:100D62003100AE31AF3290689E126EE6E493F874B1
:100D72000193900891C8F0A3C8F0D2990210DF90B5
:100D820008A6E0700AA21AB35005A21BB340028063
:100D92005C900891E0FEA3E0FF74FFBE00039F5049
:100DA20009EFC39446EE9406402B900891E0FEA30F
:100DB200E0FFEFD3946DEE94064009EFC394EEEE9C
:100DC20094064011900891E0FEA3E0FFEFD394FF58
:100DD200EE94064013900891E0FEA3E0FF9000839A
:100DE200120048E599F0800385997380119008916B
:100DF200E0FEA3E0FF900083120048E599F090081E
:100E020091126F25900891E0FEA3E0FFEFB4010676
:100E1200EEB407028003020EDA900783E0B43C02CC
:100E22008003020EDAA21AB35005A21BB34002805D
:100E320055C29C1203BD900090E09008F1F0124060
:100E42008990016FE09008A7F0900170E09008A8E7
:100E5200F0900171E09008A9F074AB900051F0128B
:100E620006DA74AA900051F09008F2E0B40105127B
:100E7200078580031208C39008F2E09000CCF0903E
:100E82000051E4F08047C29C12019C74009008A7B4
:100E9200F074009008A8F074009008A9F0900090F7
:100EA200E09008F1F012408974AB900051F0120604
:100EB200DA74AA900051F01207851208C3D29C7509
:100EC20099FB75096475080012062480FED29C7590
:100ED2004D00754C007599FB0210DF900891E0FE01
:100EE200A3E0FFEF4E7006859930752F00900891B0
:100EF200E0FEA3E0FF74016F4E701BAC2FAD30AA71
:100F020031AB32ED2BFBEC3AFA8A068B0790008369
:100F1200120048E599F0900891126F25900891E02F
:100F2200FEA3E0FF74026F4E7021AC2FAD307456F9
:100F32006D4C7006E54E64E6600280031245CB12EA
:100F42004089854E99754D00754C000210DF90085E
:100F520091E0FEA3E0FF900083120048E599F09033
:100F62000891126F25900891E0FEA3E0FFAC31AD2D
:100F7200328F028E038C068D079068E4126EE6E4CF
:100F820093F9740193FEEAD39EEB994009854E9939
:100F9200754D00754C000210DF900891E0FEA3E051
:100FA200FF900083120048E599F0900891126F2596
:100FB200900891E0FEA3E0FFEFB40006EEB4010258
:100FC20080030210DF900067E0D394C7400B9000CB
:100FD20067E0C394C8F54F801A900067E0D394632A
:100FE200400B900067E0C39464F54F800690006761
:100FF200E0F54FE54F75F002A4FFAEF08F72EF906F
:101002000083126F48EFFCE0FDEC900086126F48FF
:10101200EDFCE0FDEC2DB54F0280030210D10FEF85
:10102200900083126F48E572FFE0FCEF9000871298
:101032006F48ECFFE0FCEFC39CB54F028003021047
:10104200D1E572900085126F48E572FFE0FCEF90E7
:101052000088126F48ECFFE0FCEF2CB54F71E5728F
:10106200900089126F48E0C3954F9008DFF0E57257
:1010720090008A126F48E0C3954F9008E0F0E57245
:1010820090008D126F48E0C3954F9008E1F0E57231
:1010920090008E126F48E0C3954F9008E2F0E5721F
:1010A20090008F126F48E0C3954F9008E3F0E5720D
:1010B200900090126F48E0C3954F9008E4F012063A
:1010C200507599F975096475080012062480FE7539
:0D10D20099FF75096475080012062480FE60
:0F3CC700020C9E020D81020EDD020F50020F9BB8
:1010DF0022E54C903CD6F82828730211C490089151
:1010EF00E0FEA3E0FF900057120048E0F59990084A
:1010FF0091126F25900891E0FEA3E0FF741C6F4ED4
:10110F007003754C000211C4856D990211C49008CB
:10111F0091E0FEA3E0FF900083120048E0F599EF05
:10112F00B40107EEB40703754C00900891126F25B8
:07113F000211C4900892E0C8
:0F3CD6000210E90210EC02111702111D02114237
:10114600903D48F82828738551998067855E998077
:1011560062856099805D856499805885669980531B
:10116600856799804E8568998049856999804490FC
:101176000021E0F599803CA221B340077599FAC297
:10118600218017A219B3400575990F800B90005561
:10119600E0F599900055E4F0C2198017856A9980A8
:1011A60012856599800D856B9980087599FC800379
:0311B600754C0075
:103D480002114D02115202115702115C0211610257
:103D5800116602116B02117002117502117D0211B8
:0D3D6800A20211A70211AC0211B10211B6A6
:0B11B900900891126F258003123F8DFB
:033CE5000211C108
:1011C40022E5362559FFAE5850010E9000831200D7
:1011D40048E0F537E5362559FFAE5850010E0FBFEC
:1011E40000010E900083120048E0F538853E3AE590
:1011F40037B538058537368041E538D39537401DF6
:10120400E538C395378539F0A4FFAEF0E53A8E048E
:101214008F05FF126F07ED2537F536801DE537C3BF
:1012240095388539F0A4FFAEF0E53A8E048F05FFBA
:10123400126F07EDF4042537F53622E538D39537D8
:10124400401DE538C395378539F0A4FFAEF0E53A83
:101254008E048F05FF126F07ED2537F536801DE5E7
:1012640037C395388539F0A4FFAEF0E53A8E048F84
:1012740005FF126F07EDF4042537F5362290008937
:10128400E0B4017FE56675F00A84FF7E008F36E5E1
:101294006675F00A84ADF07C008D39753E0A755888
:1012A40005755924E536C3941150051211C58006FD
:1012B4009005B8E0F536E536C394F05008E536906D
:1012C4000078F0800674EF900078F0E56675F00A17
:1012D40084FF7E008F36E56675F00A84ADF07C00ED
:1012E4008D39753E0A75580575595AE536C39411FA
:1012F40050051211C580069005EEE0F536E53690EE
:101304000050F022900089E0B40102800302139699
:10131400E56675F00A84FF7E008F36E56675F00A8F
:1013240084ADF07C008D39753E0A755805755936C3
:10133400E536C3941150051211C580069005CAE024
:10134400F536E536C394F0500585364A8003754A70
:10135400EFE56675F00A84FF7E008F36E56675F06A
:101364000A84ADF07C008D39753E0A7558057559AF
:1013740048E536C3941150051211C580069005DC6A
:10138400E0F536E536C394F0500585364B80037599
:101394004BEF22E55E75F00484FF7E008F36E55E38
:1013A40075F00484ADF07C008D39753E04755801E8
:1013B400755900E536C3943F50051211C580069057
:1013C40001C2E0F536E53690088BF8E4F0E8A3F0C6
:1013D400900054E075F020A4FFAEF09000D4E08EAD
:1013E400048F05FF126F078D369000BCE0D3955E25
:1013F40050030214A29000E0E0D3955E4010ED90FB
:1014040001C3126F48E0F52A75290002149F900069
:10141400ABE0D3955E4043E5369001C3126F48E0DC
:10142400F537E5369001E3126F48E0F5389000E0B7
:10143400E0F404255EF5399000ABE0FE9000E0E0B6
:10144400F4042EF53AE537B53805853736800312AE
:10145400123F85362A7529008041E5369001E31252
:101464006F48E0F537E536900203126F48E0F5382F
:101474009000ABE0F404255EF5399000BCE0FE90EA
:1014840000ABE0F4042EF53AE537B5380585373678
:10149400800312123F85362A7529000215499000EF
:1014A400E3E0D3955E5011E536900243126F48E0B5
:1014B400F52A7529000215499000ACE0D3955E50D9
:1014C40043E536900223126F48E0F537E536900283
:1014D40043126F48E0F5389000ACE0F404255EF563
:1014E400399000E3E0FE9000ACE0F4042EF53AE518
:1014F40037B53805853736800312123F85362A758D
:1015040029008041E536900203126F48E0F537E583
:1015140036900223126F48E0F5389000BCE0F404E2
:10152400255EF5399000ACE0FE9000BCE0F4042E9A
:10153400F53AE537B53805853736800312123F850D
:10154400362A752900229000F4E0F53B753E1175AA
:101554005802755900AE50AF51E53B75F00FA4FD2C
:10156400ACF0EDD39FEC9E4021E53B8E048F05FF4C
:10157400126F07ED75F010A4FFAEF0E55E75F01183
:1015840084FD7C00ED2FF53C800EE55E75F0118442
:10159400FF7E00EF24F0F53C853C36E55E75F011E6
:1015A40084AFF07E008F391211C585363DAE50AF41
:1015B400519000F4E075F00FA4FDACF0EDD39FEC76
:1015C4009E4028755802755910853C361211C58500
:1015D4003D37853638AE50AF51E53B8E048F05FF5D
:1015E400126F328D39853B3A12123FE53690088BE3
:1015F400F8E4F0E8A3F0752A64752900229000F459
:10160400E0F53B753E11755802755900AE50AF5167
:10161400E53B75F00FA4FDACF0EDD39FEC9E4021AB
:10162400E53B8E048F05FF126F07ED75F010A4FFE4
:10163400AEF0E56075F01184FD7C00ED2FF53C8083
:101644000EE56075F01184FF7E00EF24F0F53C8513
:101654003C36E56075F01184AFF07E008F391211CD
:10166400C585363DAE50AF519000F4E075F00FA43F
:10167400FDACF0EDD39FEC9E4028755802755910CF
:10168400853C361211C5853D37853638AE50AF518D
:10169400E53B8E048F05FF126F328D39853B3A127C
:1016A400123FE53690088BF8E4F0E8A3F0E56A60B1
:1016B40017E56AC394FE50109000E8E0B402099064
:1016C40000D6E0D3940B5002801F90088BE0FEA359
:1016D400E0FFE56A126F1774E78E048F05FF126F3F
:1016E4000790088BECF0A3EDF09000BEE0B4045F2B
:1016F400E55E75F00484FF7E008F36E55E75F004C8
:1017040084ADF07C008D39753E047558017559001F
:10171400E536C3943F50051211C580069001C2E01E
:10172400F53690088BE0FEA3E0FFE536126F1774E0
:10173400328E048F05FF126F0790088BE0FEA3E042
:10174400FFEF2DFDEE3CFC90088BECF0A3EDF07563
:101754002A6475290022900089E0B40146E5667583
:10176400F00A84FF7E008F36E56675F00A84ADF0DA
:101774007C008D39753E0A755805755900E536C3E8
:10178400941150051211C58006900594E0F536AE0B
:1017940029AF2AE5362FFF50010E7464126F5A8E5A
:1017A400298F2A90008AE0B40146E56775F00A841F
:1017B400FF7E008F36E56775F00A84ADF07C008DFE
:1017C40039753E0A75580575596CE536C394115040
:1017D400051211C58006900600E0F536AE29AF2A41
:1017E400E5362FFF50010E7464126F5A8E298F2A2A
:1017F400900099E0B40249E569C3944175F0058409
:10180400FF7E008F36E56975F00584ADF07C008DB0
:1018140039753E05755806755900E536C39413505D
:10182400051211C58006900696E0F536AE29AF2A5A
:10183400E5362FFF50010E7464126F5A8E298F2AD9
:101844009000DBE0B4020280030218F9E55E75F053
:101854001584FF7E008F36E55E75F01584ADF07C4F
:10186400008D39753E157558037559F4E536C394E2
:101874000B50051211C58006900482E0F536E5365A
:1018840075F0FFA4FFAEF09000DCE08E048F05FF3E
:10189400126F07ED900075F0E56575F078A4FFAE62
:1018A400F074FF8E048F05FF126F078C588D5974E6
:1018B400028C068D071200398F36AC58AD5974046A
:1018C400FF126F328D39753E04755806755928E537
:1018D40036C3941D50051211C580069006C8E0F564
:1018E40036AE29AF2AE5362FFF50010E7464126F0D
:1018F4005A8E298F2A900088E0B4025DE56075F065
:1019040064A4FFAEF074081200398E5A8F5B74051C
:101914008E048F05FF126F078D36AE5AAF5B7405C8
:101924008E048F05FF126F328D39753E057558058B
:101934007559DEE536C3941350051211C58006901F
:101944000674E0F536AE29AF2AE5362FFF50010EB6
:101954007464126F5A8E298F2A9000CAE0707F90A7
:101964000054E075F00A84FF7E008F36900054E046
:1019740075F00A84ADF07C008D39753E0A75580502
:101984007559C0E536C3940E50051211C5800690F2
:101994000651E0F536E536900079F09000E9E0B4C0
:1019A400023C900054E075F00A84FF7E008F36906C
:1019B4000054E075F00A84ADF07C008D39753E0A60
:1019C4007558057559CFE536C3940E50051211C5E7
:1019D4008006900660E0F536E53690007AF02290B5
:1019E4000091E0B401179008E6E0252AFFAE2950E3
:1019F400010E9000E5E0126F5A8E298F2A9001099A
:101A0400E0B4011490010AE0A850B80004955150C4
:101A140007E55EC3955F400280139000B3E0252A7A
:101A2400FFAE2950010E8E298F2A021E4A90009182
:101A3400E0B40306A21EB3B3400280509008F0E065
:101A440070109008E9E0C39405A850B800069551B9
:101A5400400280109000B3E0252AFFAE2950010E09
:101A64008E298F2A9008F0E0600D9008E9E0A850D4
:101A7400B800069551400280109000B3E0252AFF7B
:101A8400AE2950010E8E298F2A021E4A90008BE047
:101A9400B402028003021E4A90008EE0602FE566C5
:101AA400D394464028900018E0FEA3E0FF9000C9BC
:101AB400E075F003A4FDACF0EFD39DEE9C400E90D6
:101AC40000EDE0A850B80005D395515003021E4A1A
:101AD4009000BEE0B403028003021C928560597535
:101AE4005800900095E0A850B800049551500E900D
:101AF4000096E0A858B80005D395595003021C8FEE
:101B0400E56075F002A4FFAEF074158E048F05FF36
:101B1400126F078C068D07900613120048FEE0FF33
:101B2400EE90008DE0FEEF8E0088F0A4FFAEF0741E
:101B3400648E048F05FF126F078C588D59900054E2
:101B4400E075F018A4FFAEF09000D4E08E048F0589
:101B5400FF126F078C068D0790062B120048AE58B3
:101B6400AF59E0126F1774648E048F05FF126F076C
:101B74008C588D59E564A858B80005D3955950037D
:101B8400021C06E564C39559FFE49558FE8E588FF0
:101B9400597428BE00039F500C7559287558007459
:101BA4000D900055F0AE58AF5990008EE0126F17AB
:101BB40074288E048F05FF126F078C588D59900876
:101BC4008BE0FEA3E0FF740A8E048F05FF126F07FB
:101BD4008D068C07AC58AD59CFCECF120003740AD2
:101BE4008E048F05FF126F078C588D5990088BE077
:101BF400FEA3E0FF126F6290088BEEF0A3EFF002F9
:101C04001C8FE564A858B800049559507EAE58AFAF
:101C140059E564126F5A8E588F597428BE00039F79
:101C2400500C755928755800740D900055F0AE5835
:101C3400AF5990008EE0126F1774288E048F05FF41
:101C4400126F078C588D5990088BE0FEA3E0FF7447
:101C54000A8E048F05FF126F078D068C07AC58ADF2
:101C640059CFCECF120003740A8E048F05FF126F72
:101C7400078C588D5990088BE0FEA3E0FFEF2DFDF3
:101C8400EE3CFC90088BECF0A3EDF0021E4A9000B1
:101C9400D6E0855EF0A4FFAEF07405126F177407EA
:101CA4001200398E588F59900095E0A850B800045E
:101CB40095515012900096E075F002A4FDACF0EF3F
:101CC400C39DEE9C4003021E4AE55E75F00B84FF43
:101CD4007E00900613120048FEE0FFEE90008DE0B7
:101CE400FEEF8E0088F0A4FFAEF074648E048F05BE
:101CF400FF126F078C588D59900054E075F018A4AA
:101D0400FFAEF09000D4E08E048F05FF126F078CB5
:101D1400068D0790062B120048AE58AF59E0126F9B
:101D24001774648E048F05FF126F078C588D59E564
:101D340064A858B80005D395595003021DC1E56441
:101D4400C39559FFE49558FE8E588F597428BE00E8
:101D5400039F500C755928755800740D900055F068
:101D6400AE58AF5990008EE0126F1774288E048F0E
:101D740005FF126F078C588D5990088BE0FEA3E085
:101D8400FF740A8E048F05FF126F078D068C07AC53
:101D940058AD59CFCECF120003740A8E048F05FFBD
:101DA400126F078C588D5990088BE0FEA3E0FF1248
:101DB4006F6290088BEEF0A3EFF0021E4AE564A870
:101DC40058B800049559507EAE58AF59E564126F67
:101DD4005A8E588F597428BE00039F500C75592889
:101DE400755800740D900055F0AE58AF5990008EA0
:101DF400E0126F1774288E048F05FF126F078C583A
:101E04008D5990088BE0FEA3E0FF740A8E048F05C1
:101E1400FF126F078D068C07AC58AD59CFCECF1289
:101E24000003740A8E048F05FF126F078C588D59B6
:101E340090088BE0FEA3E0FFEF2DFDEE3CFC900844
:101E44008BECF0A3EDF0229000E9E0B4027BE55EB8
:101E540075F00884FF7E008F36E55E75F00884AD6A
:101E6400F07C008D39753E087558017559E0E536EA
:101E7400C3943F50051211C58006900282E0F536E6
:101E8400E53690088DF8E4F0E8A3F090088DE0FEC4
:101E9400A3E0FFAC29AD2A12000374648E048F05FD
:101EA400FF126F0790088DECF0A3EDF0900086E030
:101EB4008C068D07126F1774648E048F05FF126FE2
:101EC4000790088DECF0A3EDF090088BE0FEA3E002
:101ED400FFAC29AD2A12000374648E048F05FF122F
:101EE4006F0790088BECF0A3EDF0900086E08C0671
:101EF4008D07126F1774648E048F05FF126F07909D
:101F0400088BECF0A3EDF0A203401DAE50AF51746A
:101F140005BE00039F5002D203E560D394CC400871
:101F2400D2017411900055F0229000E8E0B4020848
:101F34009000D6E0640B6002804590088BE0FEA31D
:101F4400E0FFE56A126F1774E78E048F05FF126FC6
:101F54000790088BECF0A3EDF09000E9E0B4021FC9
:101F640090088DE0FEA3E0FFE56A126F1774E78E18
:101F7400048F05FF126F0790088DECF0A3EDF0902D
:101F840000A8E05402601B90009FE0A850B8001223
:101F9400D39551400DA203B3B35007E560C3949A9F
:101FA4004002805FAE33AF3490009DE075F002A430
:101FB400FDACF0EF2DFDEE3CFC74022DFD50010C48
:101FC400E560BC003ED39D403A754201A2254033F2
:101FD40090009EE075F05EA4FDACF07405FF126FF6
:101FE400078C5A8D5B12495790088BE0FEA3E0FFE3
:101FF40090009EE02FFF50010E90088BEEF0A3EFAF
:10200400F0D225E560A833B8000495345002C22507
:10201400856034753300E54270030221239000FB90
:10202400E0C39542500302211590010BE0C39402D2
:1020340040030220BFE56675F00A84FF7E00900528
:1020440083120048E0F559755800AE58AF59900016
:102054009EE0126F1774648E048F05FF126F078C55
:102064005A8D5B9000FBE004C395428C068D0712E9
:102074006F179000FBE08E048F05FF126F078C5AD8
:102084008D5B90088BE0FEA3E0FFEF2DFDEE3CFCA2
:1020940090088BECF0A3EDF09000E9E0B4021A9004
:1020A400088DE0FEA3E0FFAA5AAB5BEF2BFBEE3AF0
:1020B400FA90088DEAF0A3EBF080569000FBE00460
:1020C400C39542854AF0A4FFAEF09000FBE08E0475
:1020D4008F05FF126F078C5A8D5B90088BE0FEA36F
:1020E400E0FFEF2DFDEE3CFC90088BECF0A3EDF04F
:1020F4009000E9E0B4021A90088DE0FEA3E0FFAA84
:102104005AAB5BEF2BFBEE3AFA90088DEAF0A3EBA7
:10211400F005429000FBE0C39542500375420090E5
:1021240000A8E05401601B90009CE0A850B8001285
:10213400D39551400DA203B3B35007E55EC394CCCD
:102144004002806090009AE075F003A4FFAEF0E5D1
:102154003F2FFF50010E74032FFF50010EE55EBEAA
:102164000042D39F403E754301A225403790009B17
:10217400E075F05EA4FFAEF074058E048F05FF12C7
:102184006F078C5A8D5B12495790088BE0FEA3E0D1
:10219400FF90009BE02FFF50010E90088BEEF0A300
:1021A400EFF0D225E55EC3953F5002C225855E3F20
:1021B400E54370030222BD9000FCE0C39543500345
:1021C4000222AF90010BE0C394024003022259E5BE
:1021D4006675F00A84FF7E00900583120048E0F5DE
:1021E40059755800AE58AF5990009BE0126F1774A0
:1021F400648E048F05FF126F078C5A8D5B9000FC70
:10220400E004C395438C068D07126F179000FCE021
:102214008E048F05FF126F078C5A8D5B90088BE03C
:10222400FEA3E0FFEF2DFDEE3CFC90088BECF0A349
:10223400EDF09000E9E0B4021A90088DE0FEA3E00E
:10224400FFAA5AAB5BEF2BFBEE3AFA90088DEAF04B
:10225400A3EBF080569000FCE004C39543854BF05B
:10226400A4FFAEF09000FCE08E048F05FF126F0710
:102274008C5A8D5B90088BE0FEA3E0FFEF2DFDEE02
:102284003CFC90088BECF0A3EDF09000E9E0B40284
:102294001A90088DE0FEA3E0FFAA5AAB5BEF2BFB7C
:1022A400EE3AFA90088DEAF0A3EBF005439000FCB7
:1022B400E0C39543500375430090088BE0FEA3E010
:1022C400FF9000ADE0BE00039F500D9000ADE09084
:1022D400088BF8E4F0E8A3F09000E9E0B40212906F
:1022E400088DE0FEA3E0FF9000ADE0BE00059F4036
:1022F40002800D9000ADE090088DF8E4F0E8A3F0C2
:10230400229000E9E0B401028003022453A203B343
:10231400500302243A9000B4E0B4017A90088BE0B0
:10232400FEA3E0FFAC50AD51120003743C8E048F49
:1023340005FF126F079000C4E0BC00159D40129089
:10234400088BE0FEA3E0FF9000C6E0BE00039F50B0
:1023540002D20290088BE0FEA3E0FFAC50AD511214
:102364000003743C8E048F05FF126F079000C4E0D5
:10237400C3940ABC001AD39D401690088BE0FEA3B8
:10238400E0FF9000C6E0C39405BE0004D39F500252
:102394008002C202807A90088BE0FEA3E0FFAC507A
:1023A400AD5112000374788E048F05FF126F0790ED
:1023B40000C4E0BC00159D401290088BE0FEA3E031
:1023C400FF9000C6E0BE00039F5004D202804190FB
:1023D400088BE0FEA3E0FFAC50AD5112000374780B
:1023E4008E048F05FF126F079000C4E0C3940ABCEB
:1023F400001AD39D401690088BE0FEA3E0FF9000E6
:10240400C6E0C39405BE0004D39F50028002C202FA
:10241400A202B3402190088BE0FEA3E0FF9000C528
:10242400E0126F1774648E048F05FF126F07900813
:102434008BECF0A3EDF0A202B3400CA22940067489
:1024440024900055F0D229A2024002C2298002C27F
:1024540002900050E06006A203B3B34002801990DA
:10246400088BE0FEA3E0FF900050E02FFF50010E28
:1024740090088BEEF0A3EFF0A200B34006A201B3E4
:10248400B35009900020E4F0A3F0802D90088BE075
:10249400FEA3E0FF7400D39F74019E401190088B4B
:1024A400E0F8A3E0900020C8F0A3C8F0800B74FF0C
:1024B400900020F8E4F0E8A3F09000CBE0C394048B
:1024C400400C9008EDE0C3940240030225AD900057
:1024D400B4E0B4014790088BE0FEA3E0FF745E1201
:1024E4006F1774058E048F05FF126F0790088BEC2D
:1024F400F0A3EDF09000E9E0B4021F90088DE0FE37
:10250400A3E0FF745E126F1774058E048F05FF122B
:102514006F0790088DECF0A3EDF0804590088BE0F8
:10252400FEA3E0FF745E126F17740A8E048F05FF1A
:10253400126F0790088BECF0A3EDF09000E9E0B483
:10254400021F90088DE0FEA3E0FF745E126F177403
:102554000A8E048F05FF126F0790088DECF0A3ED2F
:10256400F090088BE0FEA3E0FF7402BE000CD39F42
:102574004008752802752700800A90088BE0F5272B
:10258400A3E0F52890088DE0FEA3E0FF7402BE00EE
:102594000CD39F4008752C02752B00800A90088D7F
:1025A400E0F52BA3E0F52C804690088BE0FEA3E039
:1025B400FF7401BE000CD39F4008752801752700E5
:1025C400800A90088BE0F527A3E0F52890088DE0B9
:1025D400FEA3E0FF7401BE000CD39F4008752C01DC
:1025E400752B00800A90088DE0F52BA3E0F52C9064
:1025F400001EE527F0A3E528F0A22CB34009C20091
:10260400900020E4F0A3F022900054E090038312A1
:102614006F48E0F540754164900054E0FE9000BFBF
:10262400E0D39E4037E55E75F00884FF7E008F3668
:10263400E55E75F00884ADF07C008D39753E087553
:102644005803755996E536C3941F50051211C58079
:1026540006900438E0F5368536418035E55E75F040
:102664000884FF7E008F36E55E75F00884ADF07C4B
:10267400008D39753E087558037559B6E536C3940F
:102684001F50051211C58006900458E0F5368536B2
:1026940041229000F5E0F53B753E117558047559DB
:1026A40000AE50AF51E53B75F00FA4FDACF0EDD397
:1026B4009FEC9E4021E53B8E048F05FF126F07EDD2
:1026C40075F010A4FFAEF0E55E75F01184FD7C009A
:1026D400ED2FF53C800EE55E75F01184FF7E00EF72
:1026E40024F0F53C853C36E55E75F01184AFF07E50
:1026F400008F391211C585363DAE50AF519000F5AB
:10270400E075F00FA4FDACF0EDD39FEC9E4028756E
:102714005804755910853C361211C5853D378536E8
:1027240038AE50AF51E53B8E048F05FF126F328DEA
:1027340039853B3A12123F85364075416422900038
:10274400F5E0F53B753E11755804755900AE50AF70
:1027540051E53B75F00FA4FDACF0EDD39FEC9E402A
:1027640021E53B8E048F05FF126F07ED75F010A471
:10277400FFAEF0E56075F01184FD7C00ED2FF53CB3
:10278400800EE56075F01184FF7E00EF24F0F53CC7
:10279400853C36E56075F01184AFF07E008F391208
:1027A40011C585363DAE50AF519000F5E075F00F80
:1027B400A4FDACF0EDD39FEC9E40287558047559E8
:1027C40010853C361211C5853D37853638AE50AF7D
:1027D40051E53B8E048F05FF126F328D39853B3AEC
:1027E40012123F8536407541649000F0E0B40479DC
:1027F400900054E0FE9000BFE0D39E4037E55E7544
:10280400F00884FF7E008F36E55E75F00884ADF035
:102814007C008D39753E08755803755996E536C3A5
:10282400941F50051211C58006900438E0F53685D2
:1028340036418035E55E75F00884FF7E008F36E50D
:102844005E75F00884ADF07C008D39753E087558CE
:10285400037559B6E536C3941F50051211C5800699
:10286400900458E0F53685364122900089E0B401A1
:102874003BE56675F00A84FF7E008F36E56675F0E9
:102884000A84ADF07C008D39753E0A75580575597A
:1028940012E536C3941150051211C580069005A6A1
:1028A400E0F536E5412536C39464F54190008AE0AD
:1028B400B4013BE56775F00A84FF7E008F36E56757
:1028C40075F00A84ADF07C008D39753E0A755805A3
:1028D40075597EE536C3941150051211C5800690D2
:1028E4000612E0F536E5412536C39464F541E5402A
:1028F4002541F535900091E0B402109008E5E025FB
:1029040035FE9000E5E0F4042EF5359000E8E0D3C0
:1029140094014040E56AC394E7501D74E7C3956A87
:10292400FE9008E7E08E00F5F0E884FF7E008F3625
:10293400E5352536F535801CE56AC394E7FE900835
:10294400E7E08E00F5F0E884FF7E008F36E535C3BE
:102954009536F535A2034006E5402464F535E535A2
:10296400D394644009E535C39464F5358003753523
:10297400009000C1E0C3953550069000C1E0F535E4
:1029840022D200900077E0A850B800049551503E40
:10299400900077E0A850B800049551500375350FA6
:1029A400900077E004A850B80004955150037535A1
:1029B40007900077E02402A850B800049551500213
:1029C400C200900077E060067409900055F0C224BC
:1029D4007E017F009000C7E0126F179000D6E08E52
:1029E400048F05FF126F07E55EBC000CD39D400801
:1029F400D22C740A900055F0900089E0B40109903B
:102A040000C8E0C39566400280159000DAE0A85043
:102A1400B8000495515002C200740B900055F09018
:102A24000089E0B40107E566C394644002801D9008
:102A34000120E0600D900120E0A850B800069551F7
:102A440040028008C200740B900055F0A2004003BD
:102A5400753500C22B900109E0B4011490010AE01D
:102A6400A850B8000495515007E55EC3955F400235
:102A7400802A9000B2E0D3941D400B9000B2E0C3D2
:102A8400941EF5358003753500A22840087415900E
:102A94000055F0D22BD228D226022B7FC226C22880
:102AA400900091E0B40306A21EB3B34003022B7F4F
:102AB4009008E9E0C39405A850B800049551500665
:102AC4009008F0E06002801F9000B2E0D3941D40B3
:102AD4000B9000B2E0C3941EF53580037535007485
:102AE4000C900055F0D22B9008E9E0A850B80004EF
:102AF400955150069008F0E07002801F9000B2E0FB
:102B0400D3941D400B9000B2E0C3941EF5358003AE
:102B1400753500740C900055F0D22B9008E9E0A8AC
:102B240050B80004955150319000D0E0B40228D23E
:102B3400249008EFE0FE9008F0E0D39E5006900841
:102B4400F0E0700280099008EFE4F0C2248006905F
:102B540008EFE004F08002C2009008E9E02405A830
:102B640050B80004955150139000D0E0B4020A907C
:102B740008F0E07002D2248002C200A223B34027EE
:102B84009000B2E0D3941D400B9000B2E0C3941EB9
:102B9400F5358003753500A2274006741090005562
:102BA400F0D227D22B8002C22785356B9000B2E089
:102BB400D3941D4018900080E02535FE900054E029
:102BC40075F01E84FC7F00EE2CF5358037A22BB304
:102BD4004016900080E0FE900054E075F01E84FCE6
:102BE4007F00EE2CF535801C900082E02535FE90A8
:102BF4000080E02EFE900054E075F01E84FC7F00FF
:102C0400EE2CF535A22CB34005D224756B0022902E
:102C14000054E075F00584FF7E008F36900054E088
:102C240075F00584ADF07C008D39753E057558034B
:102C34007559D69000D4E01475F00584FF7E00E544
:102C440036BE00039F50051211C5800BE536900473
:102C540059126F48E0F536E5369008E8F09008E838
:102C6400E0FE9000C3E0C39E50089000C3E09008CB
:102C7400E8F09000B2E0D3941D401E9008E8E0FE16
:102C8400900080E02EFE900054E075F01E84FC7FDE
:102C940000EE2C9008E8F0803FA22BB3401890007F
:102CA40080E0FE900054E075F01E84FC7F00EE2C62
:102CB4009008E8F080229008E8E0FE900082E02E80
:102CC400FE900080E02EFE900054E075F01E84FC1F
:102CD4007F00EE2C9008E8F022900089E0B40136E1
:102CE400E56675F00A84FF7E00900583120048E0D3
:102CF400F545E545D394644010E545C3946475F007
:102D04000F84FF7E008F4580037545009000A6E088
:102D14002545F54580069000A6E0F54522E5667553
:102D2400F00A84FF7E00900583120048E0C3946992
:102D34004007E566D3946440559000F0E0C39403E3
:102D44005026900885E0FEA3E0FF7404120039E5E4
:102D54005E126F17740F8E048F05FF126F079008B1
:102D640083ECF0A3EDF08024900885E0FEA3E0FF5F
:102D74007404120039E560126F17740F8E048F0506
:102D8400FF126F07900883ECF0A3EDF0800F90081A
:102D940085E0F8A3E0900883C8F0A3C8F0A203403C
:102DA4001A900885E0FEA3E0FF7403126F17740104
:102DB400120039900883EEF0A3EFF0900099E0B48C
:102DC4000262E569C3944175F00584FF7E008F3685
:102DD400E56975F00584ADF07C008D39753E0575A7
:102DE4005806755914E536C3941750051211C58059
:102DF400069006AAE0F536900883E0FEA3E0FF748F
:102E04000A8E048F05FF126F07E5368C068D0712B4
:102E14006F17740A8E048F05FF126F07900883ECF6
:102E2400F0A3EDF0900883E0FEA3E0FF900889E0B2
:102E3400FCA3E0FDEDD39FEC9E400F900889E0F8E1
:102E4400A3E0900883C8F0A3C8F022E50875F00455
:102E5400A4FFAEF09006C6120048E0903CE8F828C3
:102E64002873804C85517280479000D6E0855EF0CF
:102E7400A4FFAEF074081200398F7280338560723B
:102E8400802E8566728029856772802485687280A9
:102E94001F856972801A856A728015856572801033
:102EA400856472800B856B728006900021E0F57258
:103CE800022E66022E68022E6D022E81022E860298
:103CF8002E8B022E90022E95022E9A022E9F022EB5
:073D0800A4022EA9022EAE59
:102EB400E50875F004A4FFAEF09006C7120048E5DB
:102EC4000875F004A4FFAEF0E0FC9006C8120048B8
:102ED400ECFEE0FFEEC39F4003022FBCE50875F053
:102EE40004A4FFAEF09006C6120048E0B40441E525
:102EF4000875F004A4FFAEF09006C8120048E0C3C1
:102F04009572500AE508F50CD3922D123E91E5080E
:102F140075F004A4FFAEF09006C7120048E0D39504
:102F240072400AE508F50CC3922D123E91022FBAA5
:102F3400E50875F004A4FFAEF09006C7120048E05F
:102F4400C395725015E50875F004A4FFAEF0900621
:102F5400C8120048E0D395725002800AE508F50CC7
:102F6400D3922D123E91E50875F004A4FFAEF090C3
:102F740006C7120048E0D395725015E50875F004B1
:102F8400A4FFAEF09006C8120048E0C39572500A40
:102F9400E508F50CC3922D123E919006CEE0B401E3
:102FA400099000E2E0D395605002800A7402F50CA7
:102FB400C3922D123E91806AE50875F004A4FFAE19
:102FC400F09006C7120048E0D395724015E50875E5
:102FD400F004A4FFAEF09006C8120048E0C3957256
:102FE4004002800AE508F50CC3922D123E91E508D3
:102FF40075F004A4FFAEF09006C7120048E0C39534
:10300400724015E50875F004A4FFAEF09006C812EE
:103014000048E0D39572400AE508F50CD3922D12CE
:103024003E9122AE2DAF2E74C9BE000CD39F400832
:10303400782D126F6A023141752E01752D00AE5044
:10304400AF51E545BE000DD39F40099000B8E0D3D1
:10305400954640028023754600E545C39551F572B7
:103064009000BBE0D395444008E5442572F54480C4
:10307400069000BBE0F54480020546900094E0D33E
:103084009560401CE55EC3955F4015AE50AF51E5B9
:1030940045BE00039F50099000B9E0D39547400214
:1030A400806E9008EAE0A850B8000495515003756A
:1030B40049009008EAE0A850B8000BD395514006A7
:1030C400E5519008EAF0E5497041E551C39545F5AD
:1030D40072E572D3940540037572059000BAE0C39B
:1030E40095445007E572C3954440028009E544C302
:1030F4009572F54480069000BAE0F5449000BAE079
:10310400D3954440069000BAE0F544754700800228
:103114000547E5497016900094E0C39560500DE5AD
:10312400452405A850B8000695514002800F900030
:10313400A7E0F54475490174789008EAF022AE2DB1
:10314400AF2E74E9D39F74039E4008782D126F6AE2
:103154000232FB752E01752D00754432A21F403DCD
:10316400E54675F00284AFF07E00EF4E70057544BD
:103174001980037544329000A7E075F002A4FFAEF5
:10318400F0E546BE0006D39F4002D21F05467549AE
:103194000374789008EAF07548000232E2AE50AF4A
:1031A40051E5456F4E70030232E2E545BE000DD392
:1031B4009F40099000B8E0D395464002800F7546C1
:1031C40000E549C394035003754419800DE545C3D4
:1031D4009551F572E5462572F546900094E0D39535
:1031E40060400E9008EAE0A850B80007D39551401B
:1031F40002800C05489000A7E0B54803754900E536
:1032040049B40306A203B3B34002800A0548E54863
:10321400B43C03754902E549B402299008EAE0A8E0
:1032240050B8000ED395514009E5519008EAF07565
:103234004800900094E0C395605009754800747884
:103244009008EAF0E549705A900094E0D395604004
:103254001CE55EC3955F4015AE50AF51E545BE0019
:10326400039F50099000B9E0D39547400280087548
:10327400470075444B8028E551C39545F572E572C6
:10328400D394054003757205900094E0D395604093
:1032940008E5472572F5478006E5472406F5477596
:1032A4004800E5497016900094E0C39560500DE520
:1032B400452405A850B8000695514002800375497D
:1032C40001E549B4011875441905489000A7E0B513
:1032D400480675490275480074789008EAF0A2011E
:1032E400B34003754432E54475F00AA4FFAEF09090
:1032F400088FEEF0A3EFF022E56E903D0FF828283A
:1033040073023CA890008CE0700302362C9000C23B
:10331400E0B4010280030234BF900052E0655D60B6
:1033240009E551455060030234BC7E017F00E5BECF
:10333400126F17E5BD2FFF50010E8E588F59900163
:1033440027E075F010A4FDACF08C5A8D5BEFD39D93
:10335400EE9C4009126F628E588F59800675590091
:10336400755800AE58AF59740E126F179000B7E03D
:103374008E048F05FF126F07900893ECF0A3EDF015
:10338400E56A600FE56AC394FE50089000E8E064C3
:1033940002600280649000D6E0B40B1F900893E0B2
:1033A400FEA3E0FF74E7126F17E56A8E048F05FF32
:1033B400126F07900893ECF0A3EDF09000D6E0D3E1
:1033C400940B40089000BEE064046002802B9008D7
:1033D40093E0FEA3E0FF900897E0FCA3E0FDEFD3A9
:1033E4009DEE9C400D126F62900893EEF0A3EFF0F7
:1033F4008007900893E4F0A3F0900893E0FEA3E024
:10340400FFEFD39400EE94014008D22C7426900070
:1034140055F0A22CB3B3502C7E057F009000D6E06B
:103424008E048F05FF126F07900893E0FEA3E0FF60
:10343400EFC39DEE9C400FAC50AD51740FBC000423
:10344400D39D50028002C22C90008CE0B4022790DD
:103454000895E0FEA3E0FF900893E0FCA3E0FDEFF5
:103464002DFDEE3CFC74018C068D0712003990088A
:1034740093EEF0A3EFF0900893E0FEA3E0FF900832
:1034840095E0FCA3E0FDEDD39FEC9E4004D22280A6
:1034940002B222900893E0F8A3E0900895C8F0A344
:1034A400C8F09000BEE064016006A222B3B34002FB
:1034B4008006900894E0F55E02362AD2227E017FCF
:1034C40000E5BE126F17E5BD2FFF50010E8E588F19
:1034D40059900127E075F010A4FDACF08C5A8D5B77
:1034E400EFD39DEE9C4009126F628E588F5980066F
:1034F400755900755800AE58AF59740E126F179075
:1035040000B7E08E048F05FF126F07900893ECF06C
:10351400A3EDF0E56A600FE56AC394FE50089000DD
:10352400E8E06402600280649000D6E0B40B1F906F
:103534000893E0FEA3E0FF74E7126F17E56A8E04B8
:103544008F05FF126F07900893ECF0A3EDF0900045
:10355400D6E0D3940B40089000BEE064046002807F
:103564002B900893E0FEA3E0FF900897E0FCA3E013
:10357400FDEFD39DEE9C400D126F62900893EEF028
:10358400A3EFF08007900893E4F0A3F0900893E091
:10359400FEA3E0FFEFD39400EE94014008D22C7414
:1035A40026900055F0A22CB3B3502C7E057F0090DA
:1035B40000D6E08E048F05FF126F07900893E0FE9B
:1035C400A3E0FFEFC39DEE9C400FAC50AD51740FD0
:1035D400BC0004D39D50028002C22C90008CE0B445
:1035E4000227900895E0FEA3E0FF900893E0FCA377
:1035F400E0FDEF2DFDEE3CFC74018C068D071200FE
:1036040039900893EEF0A3EFF0900893E0F8A3E06C
:10361400900895C8F0A3C8F09000BEE0640160066D
:10362400900894E0F55E8003755E00900088E07079
:1036340006756E030232FC75BB18023CA8023CA856
:10364400900088E070030237B57E017F00E5BE126A
:103654006F17E5BD2FFF50010E8E588F599000CE85
:10366400E0B4010F7E0F7FFFAC58AD59126F628E2C
:10367400588F599000F3E0B40245AE58AF5990000A
:103684002AE0FCA3E0FDEDD39FEC9E400A90002AC3
:10369400E558F0A3E559F0AE58AF5990002CE0FC82
:1036A400A3E0FDEFD39DEE9C400A90002CE558F07A
:1036B400A3E559F0AE58AF5974041200398F6090E5
:1036C40000F3E0704CAE58AF5990002AE0FCA3E040
:1036D400FDEFD39DEE9C4009126F628E588F598086
:1036E40006755900755800AE58AF597410126F170B
:1036F4009000F2E08E048F05FF126F078C588D59ED
:1037040074FFBC0009D39D40058559608003756032
:10371400FE9000BEE0B4010280030237B3A203B3FB
:10372400B3500E900092E0A850B80005D3955150C4
:103734000280719000CFE08560F0A4FFAEF0746465
:103744008E048F05FF126F078C588D59E56A601639
:10375400E56AC394FE500F9000E8E0B402089000BC
:10376400D6E0640B60028017AE58AF5974E7126F4D
:1037740017E56A8E048F05FF126F078C588D59AEBA
:1037840058AF59900893E0FCA3E0FDEDD39FEC9E65
:10379400400585595E800BA222B34006900894E050
:1037A400F55E800BA222B34006900894E0F55E809B
:1037B4000375600090008BE07006756E050232FCA4
:1037C40075BB19023CA8023CA890008BE070030270
:1037D400389CE55DD3955C400302389A900028E05C
:1037E400FEA3E0FFE564126F5A900028EEF0A3EF09
:1037F400F09000F8E0B402247E017F00E5BE126F71
:1038040017E5BD2FFF50010E8F048E057E0F7FFF3D
:10381400CDCCCD126F628E588F5980147E017F00FB
:10382400E5BE126F17E5BD2FFF50010E8E588F595C
:103834009000F8E07017AE58AF59740A126F1774FD
:10384400518E048F05FF126F078D648019AE58AF37
:1038540059740A126F178F048E057E017F95CDCCA3
:10386400CD126E058F64E564D3946440037564647B
:10387400900028E0FEA3E0FFE5642FFF50010E90C6
:103884000028EEF0A3EFF090008FE0048E048F0583
:10389400FF126F078D6480037564329000DBE07063
:1038A40006756E070232FC75BB13023CA8023CA8E5
:1038B4009000DBE0604A7E017F00E5BE126F17E5F1
:1038C400BD2FFF50010E8E588F5974041200398F8A
:1038D400659000DDE08565F0A4FDACF07464FF1232
:1038E4006F078D659000DCE08565F0A4FFAEF07491
:1038F400FF8E048F05FF126F07ED900076F08003B2
:10390400756500900089E07006756E090232FC75D9
:10391400BB17023CA8023CA8900089E0B4010280D5
:10392400030239B07E017F00E5BE126F17E5BD2F9B
:10393400FF50010E8E588F599008EBE060199008E3
:10394400EBE01490692A12008CE493FC740193FD5B
:10395400EDC39FEC9E400280069008EBE014F090CB
:1039640008EBE0C394B3501DAE58AF599008EBE098
:103974000490692A12008CE493FC740193FDEFC354
:103984009DEE9C400280069008EBE004F09008EB6A
:10399400E0FE9000AFE08E0088F0A4FFAEF0746407
:1039A4008E048F05FF126F078D6680037566009085
:1039B400008AE07006756E0B0232FC75BB16023C81
:1039C400A8023CA890008AE0B401028003023A5C99
:1039D4007E017F00E5BE126F17E5BD2FFF50010E7B
:1039E4008E588F599008ECE060199008ECE0149020
:1039F4006A9412008CE493FC740193FDEDC39FEC74
:103A04009E400280069008ECE014F09008ECE0C3BD
:103A140094B3501DAE58AF599008ECE004906A94EA
:103A240012008CE493FC740193FDEFC39DEE9C4063
:103A34000280069008ECE004F09008ECE0FE9000B0
:103A4400B5E08E0088F0A4FFAEF074648E048F0598
:103A5400FF126F078D67800375670075BB1F023CFB
:103A6400A8023CA87E017F00E5BE126F17E5BD2FBA
:103A7400FF50010E8E588F597409126F1774E68E19
:103A8400048F05FF126F078D69900091E070067531
:103A94006E0F0232FC75BB15023CA8023CA89000D4
:103AA40091E07003023BF37E017F00E5BE126F17C5
:103AB400E5BD2FFF50010E8E588F59740412003942
:103AC4008F68900091E0B401159000E5E08568F0FE
:103AD400A4FFAEF07407120039EF9008E6F09000EE
:103AE40091E0B402159000E5E08568F0A4FFAEF023
:103AF4007407120039EF9008E5F0900091E0B403E8
:103B0400028003023BD69000D2E07052E568C39471
:103B140019500FD21E9000B1E09008E9F09008EE21
:103B2400E4F0E568D394644004A21E4002802D9022
:103B340008EEE004F09008EEE0FE900124E0B50603
:103B44000B9008E9E004F09008EEE4F09008E9E056
:103B540064966006900124E07002C21E80639000A7
:103B6400B1E070349000E5E08568F0A4FFAEF07435
:103B7400FF8E048F05FF126F07ED9008E9F0AE5039
:103B8400AF51741EBE0006D39F4002D21EE560D31F
:103B940094E54002C21E8029E568C3940A500DAE24
:103BA40050AF51741EBE0004D39F50028002D21E37
:103BB400E560D394E54002C21E9000B1E09008E9AC
:103BC400F09008E9E0C39405500674059008E9F004
:103BD400C223900091E0B40414E568C39419500220
:103BE400D223E568D394324002C223C21E800375F7
:103BF40068009000E8E07006756E110232FC75BB37
:103C040014023CA8023CA89000E8E07003023C9532
:103C14007E017F00E5BE126F17E5BD2FFF50010E38
:103C24008E588F59900128E075F010A4FDACF08CEB
:103C34005A8D5BEFD39DEE9C4009126F628E588FB4
:103C4400598006755900755800AE58AF59740E1254
:103C54006F179000EFE08E048F05FF126F078C5AE8
:103C64008D5B74FFBC00039D5005756AFF8003855E
:103C74005B6AE56A75F00BA4FFAEF09000D6E08EA7
:103C8400048F05FF126F07900897ECF0A3EDF08006
:103C940003756A0090008CE0600575BB1A8003759B
:043CA400BB188000C9
:103D0F000233050233080236410236440237CA0233
:103D1F0037CD0238B10238B402391902391C0239D1
:103D2F00C50239C8023A65023A68023A9F023AA2BE
:093D3F00023C08023C0B023CA806
:103CA800E56E75F00284AFF07E00EF4E7002D2EC44
:033CB800056E2274
:096F48002582F582500205832226
:0F008C0025E050020583258250020583F582226C
:106EE600EF2F500205832582F582E5833E2EF5833A
:016EF6002279
:106F5A00CFC39FFF50011E22C3EF9DFFEE9CFE226E
:086F6A000806B6000218062219
:0D6F2500A3E004F07006126F3EE004F022BD
:0E003900048007C3CE13CECF13CFD5E0F6223E
:106E0500BC000FBE0008ED8FF084FFADF022E4FE5C
:106E1500FF22BE000DEF60FE54F0606F20E7030215
:106E25006EBBEAC0E0EBC0E078017A0075F001EED8
:106E350020E710EF25E0FFEE33FE0AC5F023C5F08D
:106E450030E7F0EA5407F9096A7A007B0060010827
:106E5500C3EC9E40167004ED9F4010ED9FFDEC9E27
:106E6500FCE5F0CA4ACA03F5F08005E5F003F5F044
:106E7500C3EE13FEEF13FFD9D77908CACBCAD8D012
:106E8500EAFEEBFFD0E0FBD0E0FA22EC8FF084FCC9
:106E9500ED54F045F0C48FF084FEEDC454F045F098
:106EA500C48FF084FDEEC4FE54F02DFFEE540F3C6C
:106EB500FEADF07C0022790078008FF0EC7E082092
:106EC500E70DC3CD33CD33C933C9C833C8DEF0842C
:106ED50049F9E5F08FF0BE00E6FD7C00E9FFE8FE2C
:016EE500228A
:0E6F1700F88FF0A4FFE5F0CE88F0A42EFE2245
:10000300EF8DF0A4F9A8F0EF8CF0A428F8EE8DF0B2
:06001300A428FEE9FF2213
:106EF700600D782B026F01007830D8FED5E0F822BC
:106F0700EEC0E07E00126E05EFFDEEFCD0E0FE2243
:0C6F3200EEC0E07E00126E05D0E0FE22F2
:03001B0002001EC2
:0300530002005652
:03009B00020071EF
:03000000026F513B
:096F510075817475D000024A94A8
:0B004800E5822FF582E5833EF5832260
:0A6F3E000582D58202158315822218
:10001E00C0E0C0F0C083C082C0D075D000124A1CB0
:0B002E00D0D0D082D083D0F0D0E032E0
:10005600C0E0C0F0C083C082C0D075D000124A1F75
:10006600D0D0D082D083D0F0D0E032C0E0C0F0C093
:1000760083C082C0D075D000124A4ED0D0D082D074
:0600860083D0F0D0E0324F
:00000001FF
